:020000040000FA
:100000000C9468030C9490030C9490030C9490034C
:100010000C9490030C9490030C9490030C94900314
:100020000C9490030C9490030C9490030C94900304
:100030000C9490030C9490030C9490030C949003F4
:100040000C9481250C9490030C944F250C94292535
:100050000C9490030C9490030C9490030C949003D4
:100060000C94CB250C94900307634236B79BD8A71A
:100070001A39685618AEBAAB558C1D3CB7CC5763CD
:10008000BD6DEDFD753EF6177231BF000000803F7B
:1000900008000000BE922449123EABAAAA2ABECD97
:1000A000CCCC4C3E00000080BEABAAAAAA3E000009
:1000B0000000BF000000803F000000000008417801
:1000C000D3BB4387D1133D190E3CC3BD4282AD2B38
:1000D0003E68EC8276BED98FE1A93E4C80EFFFBE30
:1000E00001C4FF7F3F00000000004E414E494E49D1
:1000F0005459494E46CDCCCC3D0AD7233C17B7D1F5
:100100003877CC2B329595E6241FB14F0A0000209A
:10011000410000C84200401C4620BCBE4CCA1B0E19
:100120005AAEC59D7400407A10F35A00A0724E1862
:10013000090010A5D4E80000E87648170000E40B99
:1001400054020000CA9A3B000000E1F5050000805F
:10015000969800000040420F000000A086010000B9
:1001600000102700000000E8030000000064000009
:100170000000000A00000000000100000000002C48
:1001800076D888DC674F0823DFC1DFAE59E1B1B70D
:1001900096E5E3E453C63AE651997696E8E6C284DA
:1001A00026EB898C9B62ED407C6FFCEFBC9C9F40F2
:1001B000F2BAA56FA5F490055A2AF75C936B6CF917
:1001C000676DC11BFCE0E40D47FEF520E6B500D0ED
:1001D000ED902E0300943577050080841E08000002
:1001E000204E0A000000C80C333333330F986E12D0
:1001F000831141EF8D2114893BE65516CFFEE6DBD6
:1002000018D1844B381BF77C1D901DA4BBE424201F
:100210003284725E228100C9F124ECA1E53D270100
:10022000080D00FE09016102CD207FFE0BFE09FED4
:100230000D00803219898080808080808000802835
:1002400043839090901367874848FC48FC484812C5
:1002500059892078A0A0702828F02012698944A428
:1002600048101020485488126787609090609488E6
:1002700074381383808080323989204040808080A8
:100280004040202239898040402020204040801674
:1002900065854830FC30481455852020F820201111
:1002A0004383706080165181F821338340E040021F
:1002B0007989020204081020408080126989304840
:1002C000848484848448301259892060A0202020AE
:1002D0002020F81269897884840408304080FC1258
:1002E0006989FC04081038040484781269890818A4
:1002F00028488888FC0808126989FC8080B8C404F2
:1003000004847812698938408080B8C48484781263
:100310006989FC0408101020204040126989788403
:10032000848478848484781269897884848C7404C1
:1003300004087021388840E040000040E040114847
:1003400088207020000070608022598908102040A9
:100350008040201008146484FC0000FC125989803D
:100360004020100810204080126989788484040895
:10037000101000101269897884849CA4AC94807851
:100380001269893048848484FC848484126989F0E9
:10039000888488F0888488F01269897884808080D5
:1003A00080808478126989F088848484848488F0C9
:1003B000126989FC808080F0808080FC126989FC51
:1003C000808080F08080808012698978848080803D
:1003D0009C848C7412698984848484FC84848484DD
:1003E000125989F820202020202020F81279893EF7
:1003F0000808080808088870126989848890A0C0D5
:10040000A09088841269898080808080808080FCB0
:100410000279898282C6AA92928282821269898432
:1004200084C4A4948C8484841269897884848484A8
:1004300084848478126989F8848484F88080808038
:10044000116A8A788484848484A4947804126989E3
:10045000F8848484F8A090888412698978848080E4
:100460007804048478027989FE101010101010109E
:1004700010126989848484848484848478027989CC
:100480008282444444282828100279898282828208
:10049000929292AA44027989828244281028448246
:1004A0008202798982824428101010101012698902
:1004B000FC04081020408080FC224989F080808064
:1004C00080808080F00279898080402010080402BA
:1004D00002124989F010101010101010F0185383F8
:1004E000205088017181FE3A22828040126686780F
:1004F000047C848C74126989808080B8C48484C42C
:10050000B81266867884808084781269890404042D
:10051000748C84848C741266867884FC808478124F
:10052000698938444040F8404040401068887488E9
:10053000887080788478126989808080B8C48484C7
:10054000848412588820006020202020F8105A8AC5
:100550000800180808080888887012698980808057
:100560008890E090888412598960202020202020E3
:1005700020F8027686EC9292929282126686B8C435
:10058000848484841266867884848484781068885D
:10059000B8C484C4B8808080106888748C848C74DB
:1005A000040404126686B8444040404012668678CF
:1005B00084601884781268884040F840404044388D
:1005C000126686888888888874125686888888503B
:1005D000502002768682829292AA441266868448CD
:1005E000303048841068888484848C740484781241
:1005F0006686FC08102040FC22598938404020C003
:1006000020404038321989808080808080808080BE
:10061000125989E010102018201010E01853834858
:10062000A890FF4C4F470056455200FFE0FFD1AF66
:10063000FF32FFD1FFFEFFE0FFD1AEFFD1FFFEFF93
:10064000E0FFD11000FFFEFFD0FFE0FFC1FFD1AE01
:10065000D580A81FD300408D142002A1C8DA0281E2
:10066000CFD9F1DB402EA4A6AFFFD0FFFE000000E3
:1006700000240027002A0000000000250028002B8D
:10068000005245420000000000230026002900041B
:100690000404040404040402020202020203030329
:1006A0000303030102040810204080010204081023
:1006B00020010204081020000000080002010000D0
:1006C000030407000000000000000000EA265F2C81
:1006D00011241FBECFEFD8E0DEBFCDBF13E0A0E0F6
:1006E000B1E0E4E0F3E702C005900D92A830B10755
:1006F000D9F726E0A8E0B3E001C01D92A436B20706
:10070000E1F713E0C7E6D3E004C02197FE010E94A1
:10071000F235C636D107C9F70E9462280C947539A4
:100720000C940000089580E008958091280690912F
:100730002906009739F120913B06FC01211123C0C5
:100740003596E491E0933C06FC013C96E491E093FD
:100750003D0680913C06082E000C990B20913D0629
:10076000821B910927FD939520913E06203441F08C
:10077000829FC001112426E0969587952A95E1F77E
:1007800080933F060895213039F43F96E491E09339
:100790003C06FC017096DACF3D96E491E0933C066E
:1007A000FC013E96D3CF089508950895AF92BF926D
:1007B000CF92DF92EF92FF920F931F93CF93DF932D
:1007C0006C017B018B01040F151FEB015E01AE185C
:1007D000BF08C017D10759F06991D601ED91FC917E
:1007E0000190F081E02DC6010995892B79F7C501AB
:1007F000DF91CF911F910F91FF90EF90DF90CF90FD
:10080000BF90AF900895CF93DF93FC014481558151
:100810006081718180E994E00E94D603EC0142E09E
:1008200050E062E671E080E994E00E94D6038C0F0C
:100830009D1FDF91CF910895FC01538D448D252F8D
:1008400030E0842F90E0821B930B541710F0CF966A
:10085000089501970895FC01918D828D981761F09C
:10086000A28DAE0FBF2FB11D5D968C91928D9F5FB3
:100870009F73928F90E008958FEF9FEF0895FC0192
:10088000918D828D981731F0828DE80FF11D858D45
:1008900090E008958FEF9FEF0895FC01918D228DD8
:1008A000892F90E0805C9F4F821B91098F7399275D
:1008B000089580E994E00E944D0421E0892B09F419
:1008C00020E0822F089580E090E0892B29F00E949B
:1008D000590481110C9400000895FC01A48DA80F07
:1008E000B92FB11DA35ABF4F2C91848D90E0019672
:1008F0008F739927848FA689B7892C93A089B18992
:100900008C91837080648C93938D848D981306C032
:100910000288F389E02D80818F7D80830895EF9296
:10092000FF920F931F93CF93DF93EC0181E0888FA9
:100930009B8D8C8D98131AC0E889F989808185FF79
:1009400015C09FB7F894EE89FF896083E889F9891B
:1009500080818370806480839FBF81E090E0DF911D
:10096000CF911F910F91FF90EF900895F62E0B8D70
:1009700010E00F5F1F4F0F731127E02E8C8D8E112B
:100980000CC00FB607FCFACFE889F989808185FF92
:10099000F5CFCE010E946D04F1CFEB8DEC0FFD2F52
:1009A000F11DE35AFF4FF0829FB7F8940B8FEA894D
:1009B000FB8980818062CFCFCF93DF93EC01888D5C
:1009C0008823B9F0AA89BB89E889F9898C9185FDCA
:1009D00003C0808186FD0DC00FB607FCF7CF8C9158
:1009E00085FFF2CF808185FFEDCFCE010E946D049F
:1009F000E9CFDF91CF910895833081F028F48130E1
:100A000099F08230A9F008958730A9F08830C9F0B4
:100A10008430B1F4809180008F7D03C0809180008C
:100A20008F7780938000089584B58F7784BD089573
:100A300084B58F7DFBCF8091B0008F778093B0001D
:100A400008958091B0008F7DF9CFCF93DF93E6ECCE
:100A5000F6E08491E2EBF6E0D491EEE9F6E0C491A1
:100A6000CC23A1F081110E94FC04EC2FF0E0EE0FEA
:100A7000FF1FEB57F94FA591B491EC91ED2381E065
:100A800090E009F480E0DF91CF91089580E090E05C
:100A9000FACF1F93CF93DF93282F30E0F901E95469
:100AA000F94F8491F901ED55F94FD491F901E157CE
:100AB000F94FC491CC23A9F0162F81110E94FC0498
:100AC000EC2FF0E0EE0FFF1FE958F94FA591B4911C
:100AD0008FB7F894EC91111108C0D095DE23DC9308
:100AE0008FBFDF91CF911F910895DE2BF8CFCF9369
:100AF000DF9390E0FC01ED55F94F24918157994F18
:100B0000FC0184918823D1F090E0880F991FFC01AB
:100B1000E359F94FA591B491FC01E958F94FC591FA
:100B2000D49161110EC09FB7F8948C91E22FE0959B
:100B30008E238C932881E223E8839FBFDF91CF919E
:100B400008958FB7F894EC91E22BEC938FBFF6CF1A
:100B50008E3008F08E5020910E0190E4299F900174
:100B600011248770822B80937C0080917A008064AE
:100B700080937A0080917A0086FDFCCF8091780086
:100B80009091790008953FB7F8948091080490916E
:100B90000904A0910A04B0910B0426B5A89B05C0D6
:100BA0002F3F19F00196A11DB11D3FBFBA2FA92FEC
:100BB000982F8827BC01CD01620F711D811D911DE9
:100BC00042E0660F771F881F991F4A95D1F7089555
:100BD0008F929F92AF92BF92CF92DF92EF92FF924D
:100BE0006B017C010E94C3054B015C01C114D1045F
:100BF000E104F104B9F00E94C305681979098A0972
:100C00009B09683E73408105910580F321E0C21A7B
:100C1000D108E108F10888EE880E83E0981EA11C37
:100C2000B11CE4CFFF90EF90DF90CF90BF90AF90DA
:100C30009F908F9008958F929F92AF92BF92CF9284
:100C4000DF92EF92FF920F931F93CF93DF938AE08F
:100C5000A82EB12CD0E0C0E0EE24EA9493E0F92E67
:100C600088248A9423E0922ED12CC12C10E000E03D
:100C70008FE00E94A8050817190790F1C816D90639
:100C800008F46C018815990568F18E159F0508F424
:100C90007C01C80FD91F65E070E080E090E00E9401
:100CA000E80581E0A81AB10819F70C0D1D1DCE0149
:100CB000801B910B8E199F098819990966E070E0D5
:100CC0000E94DE35CB01DF91CF911F910F91FF90F4
:100CD000EF90DF90CF90BF90AF909F908F9008954E
:100CE0008C01D0CF4C01D5CF8F929F92AF92BF9203
:100CF000EF92FF921F93CF93DF93C82F10921A06A3
:100D000010921B0610921C0610921D0610921E06D1
:100D100061E08FE00E94770560E08FE00E94490566
:100D20006C2F70E090E080E00E94E80560E08FE0CA
:100D30000E9477058BE990E00197F1F7C0E9D1E0D7
:100D40000E942505892B71F42197D1F78EEF9FEF33
:100D5000DF91CF911F91FF90EF90BF90AF909F9048
:100D60008F900895C0E9D1E00E942505019719F4FC
:100D70002197D1F7EBCFD8E2C0E810E090E9E92E57
:100D8000FF24F3940E942505892B29F481E0E81AB9
:100D9000F108C1F7DBCF0E94C3054B015C0180E97C
:100DA000E82EFF24F3940E942505019729F481E0A1
:100DB000E81AF108C1F7CACF0E94C305681979097A
:100DC0008A099B09693271058105910538F0E12F87
:100DD000F0E0EE5EF94F80858C2B8087C69511F48C
:100DE0001F5FC0E8D15051F690E080E0B1CF2FB73F
:100DF000F894609104047091050480910604909128
:100E000007042FBF08952091E003260F3327331FD7
:100E100021323105ECF420916604FC0190E080E081
:100E2000243069F082E00895A091E0032191AC01A3
:100E300040545C4FA40FB52FB11D2C93019686171B
:100E400098F38091E003680F6093E00380E00895D9
:100E500081E008951092660481E080936504109209
:100E6000400461E082E10E94490561E083E10E9463
:100E70004905E9EBF0E080818E7F808380818D7F62
:100E8000808388E48093B80085E48093BC00089553
:100E900010921F0410921E0410926D0410928F0481
:100EA0000E942A0783ED93E090931D0480931C0415
:100EB00084ED93E090931B0480931A040895CF93DC
:100EC000DF9391E09093BF038823B9F0C091B800FD
:100ED000D091BA008091BC008A7B8093BC0060E016
:100EE00082E10E94490560E083E10E9449050E9479
:100EF0002A07D093BA00C093B800DF91CF9108952C
:100F0000CF92DF92EF92FF920F931F93CF93DF93D5
:100F1000D0918F0481E0D13208F09CC0C0918E0442
:100F20000E94C3056B017C018091660481116CC035
:100F300082E08093660481E0809365048FEF809364
:100F4000640410926304D0936204AEE6B4E0E2E479
:100F5000F4E080E0D8138DC01092410480914104E8
:100F6000CC0FC82BC093410480914004813009F01C
:100F700084C0109240040E94C3056B017C018091E3
:100F800041048093BB008091680490916904A09112
:100F90006A04B0916B04892B8A2B8B2BA1F00E94E1
:100FA000C305009168041091690420916A0430918E
:100FB0006B046C197D098E099F090617170728070E
:100FC000390708F442C08091BC0083FDD8CF85EC7E
:100FD0008093BC000E94C3056B017C018091660474
:100FE000823009F44CC0809164048F3F09F469C0D9
:100FF00080916404803209F466C080916404803377
:1010000009F463C084E026C080916804909169046B
:10101000A0916A04B0916B04892B8A2B8B2B09F465
:1010200083CF0E94C3050091680410916904209148
:101030006A0430916B046C197D098E099F090617AB
:1010400017072807390708F06FCF809167040E94BF
:101050005F0785E010926D0410928F0410926C046B
:10106000DF91CF911F910F91FF90EF90DF90CF9084
:1010700008959D9191938F5F6DCF85EEA9CF80915B
:10108000680490916904A0916A04B0916B04892B63
:101090008A2B8B2B09F4A2CF0E94C3050091680410
:1010A0001091690420916A0430916B046C197D09D8
:1010B0008E099F09061717072807390708F08ECFF2
:1010C000C4CF80E0C7CF82E0C5CF83E0C3CFCF924B
:1010D000DF92EF92FF920F931F93CF93DF93D82F5E
:1010E000C62F613208F098C00E94C3056B017C01D5
:1010F0008091660481116BC081E0809366048093C7
:1011000065049FEF90936404109263049C0F909386
:1011100062048093410480914104DD0FD82BD09369
:10112000410480914004813009F078C0109240045D
:101130000E94C3056B017C01809141048093BB0038
:101140008091680490916904A0916A04B0916B0445
:10115000892B8A2B8B2BA1F00E94C3050091680478
:101160001091690420916A0430916B046C197D0917
:101170008E099F09061717072807390708F448C082
:101180008091BC0083FDD8CF85EC8093BC000E9489
:10119000C3056B017C0180916604813009F440C075
:1011A000809163048C1710F4C0916304E2E4F4E0CE
:1011B000A0E2B4E080E08C1355C08C2FDF91CF917A
:1011C0001F910F91FF90EF90DF90CF900895809145
:1011D000680490916904A0916A04B0916B04892B12
:1011E0008A2B8B2B09F484CF0E94C30500916804DD
:1011F0001091690420916A0430916B046C197D0987
:101200008E099F09061717072807390708F070CFBE
:10121000809167040E945F07C0E0CFCF85EEB5CF15
:101220008091680490916904A0916A04B0916B0464
:10123000892B8A2B8B2B09F4AECF0E94C30500911A
:1012400068041091690420916A0430916B046C1950
:101250007D098E099F09061717072807390708F027
:101260009ACFD6CF91919D938F5FA5CF0895E091AE
:101270001F0480911E04E81730F4F0E0E05EFB4F9D
:10128000808190E008958FEF9FEF089590911F0463
:1012900080911E042FEF3FEF981748F4E92FF0E0FC
:1012A000E05EFB4F208130E09F5F90931F04C901F7
:1012B000089580911E0490911F04891B990B089535
:1012C000CF92DF92EF92FF920F931F93CF93DF9312
:1012D0007C01CB018A0120916C04222389F0EB016F
:1012E0006B01C40ED51ECC15DD0569F06991D701DF
:1012F000ED91FC910190F081E02DC7010995F3CFAC
:10130000642F0E940307C801DF91CF911F910F91B5
:10131000FF90EF90DF90CF900895CF93DF931F92CF
:10132000CDB7DEB7698320916C042223F9F02091B8
:101330008F04203258F021E030E0FC013383228317
:1013400090E080E00F90DF91CF91089580916D043F
:10135000E82FF0E0E259FB4F998190838F5F8093F3
:101360006D0480938F0481E090E0ECCF61E0CE01CA
:1013700001960E940307F7CF80E00895DC011696DE
:10138000ED91FC91179712968C91481B477081E064
:1013900090E001C0880F4A95EAF7E60FF11D308111
:1013A000222319F0832B8083089580958323FBCF1C
:1013B000FB014181DC0112962C911297421768F0D3
:1013C00013962C911397241740F0608115962C9159
:1013D000621718F424810C94BE090895FC018081E1
:1013E0009281980F92832181921760F494819F5F7C
:1013F00094839381890F821710F08FEF820F83837C
:1014000081E0089580E00895FC011282808181507E
:10141000838314820895DB01ED91FC910994CF93AD
:10142000DF931F92CDB7DEB79E012F5F3F4F47E49A
:101430000E940B0A89810F90DF91CF910895CF937D
:10144000DF931F92CDB7DEB79E012F5F3F4F46E47B
:101450000E940B0A89810F90DF91CF910895BF926E
:10146000CF92DF92EF92FF920F931F93CF93DF9370
:101470008C01D42EE901FB01E280F380F2E34F17E7
:1014800009F476C0F417C8F08CE2481709F470C06C
:10149000EDE24E17E9F0F7E14F1779F19E014D2D7E
:1014A000B701C801DF91CF911F910F91FF90EF908D
:1014B000DF90CF90BF900C940B0A86E4481709F494
:1014C0004CC0E7E44E1709F44EC0FBE34F13E6CFE0
:1014D000B701C8010E940F0AC980C094C80EB701A5
:1014E000C8010E941F0A98819095890F8883C9823C
:1014F0008B818E5F83708B834BC047E1B701C8013E
:101500000E940B0AB701C8010E941F0ABA80B0945A
:10151000B80EB701C8010E941F0AD880D094D80E17
:10152000B701C8010E940F0ACB80C094C80EB70152
:10153000C8010E940F0A99819095890FB882C982CB
:10154000DA828B8381E0DF91CF911F910F91FF9021
:10155000EF90DF90CF90BF900895B701C8010E942F
:101560001F0A8883EFCFB701C8010E940F0AF9CF85
:10157000B701C8010E940F0AC980C094C80EB70104
:10158000C8010E941F0A98819095890F8883C9829B
:101590009E014D2DB701C8010E940B0AD3CFCF93F6
:1015A000DF93EC016A817B810E941F0A88836A8134
:1015B0007B81CE010E940F0A89836A817B8130E0A2
:1015C00020E048E4CE010E940B0A8B879E012D5C2F
:1015D0003F4F6A817B8147E1CE01DF91CF910C942F
:1015E0000B0ACF93DF93C0912606D0912706E09196
:1015F0005506F091560682E0099530E020E04AE079
:10160000BE0184E296E00E940B0AC82FE0915506C5
:10161000F091560683E00995E0915506F091560643
:1016200080E00995CC2329F084E296E00E94CF0A5D
:10163000C1E08C2FDF91CF910895FC01808D8F5FE9
:1016400008950B96FC01849108950A96FC018491FB
:101650000895FC01849108950E94290B882321F0AC
:10166000823011F083E0089586E00895FC01E60FD2
:10167000F11D849190E0982F88273196E4918E0F88
:10168000911D089568E00C94360B66E00C94360BBF
:101690005F926F927F928F929F92AF92BF92CF9202
:1016A000DF92EF92FF920F931F93CF93DF93EC01A2
:1016B000E62EF42EC22E0C811D81C8010E94290B3A
:1016C000D82E8C819D810E942C0B982E21E0AA247B
:1016D000AA94D21202C02FE0A22E8C819D810E947A
:1016E000250BD82E8C819D810E94210BB82E8C81D8
:1016F0009D810E94420BE0E6EC1578F4009769F0BA
:10170000080F191F91E6D92EBC14C0F4188A1B8A41
:101710001C8A198A1A8A80E0A0C08C819D810E944F
:10172000450BF0E4FC1538F4009729F0080F191F59
:1017300081E4D82EE9CF0F5E1F4FE6CFBD1430F302
:10174000892D90E0F80124912F3F31F40F5F1F4F56
:10175000BD14E1F2D394F6CFCD1072C08C819D817F
:101760000E94290B98012F5F3F4FF801882319F041
:10177000823009F04EC084918B8BF90124912C8B1F
:10178000F8013396E491E88BF8013496E491E98B03
:10179000F8013596E491EA8B0115110509F4BBCFE8
:1017A0008C819D810E942C0B3C89F31A9A89F91A2D
:1017B0009FEF930F9F0D2CA94EA94F1508F449C018
:1017C000921718F49F1508F047C02B899989E90EE4
:1017D0009FEF920F9E0D4BA95DA95E1508F44DC0B9
:1017E000941718F49E1508F037C0080F111D295FD3
:1017F000722E7694769476946F2C630E5E01FCE1E3
:10180000AF0EB11C872C912CF61431F15E2C6801BF
:101810004AC08491982F9F7092509A8B82958F70B6
:10182000898BF9012491822F8F708C8B22952F70D8
:101830002B8BF8013296E491E295EF70E88BACCFF8
:101840003296E491EA21E80FF92FF11D0E0F1F1FC8
:101850007FCF921708F0B6CF8889DF91CF911F9183
:101860000F91FF90EF90DF90CF90BF90AF909F903F
:101870008F907F906F905F900895941708F0B2CF8B
:10188000EBCFF60184916A817B815C8EFD8E1F8E89
:101890008E8F95014BE3CE010E940B0AFFEFCF1A0A
:1018A000DF0A28E0520E8C2D801B871550F3080D9F
:1018B000191DF394A9CF2EE93FE0009709F408958C
:1018C000F9013197F1F70197F8CFCF93DF9300D06B
:1018D000CDB7DEB720ED37E03A8329839091BC0085
:1018E000982311F081E00FC029813A81232B81F4E4
:1018F0008091190481FDF6CF8091180481110DC0EB
:1019000091E0909318040F900F90DF91CF9108957C
:1019100029813A8121503109DFCF80E0F4CF84EA78
:101920008093BC0061E080E80E94650C811102C0D8
:1019300080E008958091B900887F883051F080312F
:1019400041F0809118048111F3CF82E08093180454
:10195000EFCF88E78093BB0084E88093BC0062E00F
:1019600080E80E94650C882319F38091190481FD99
:1019700005C08091B900887F883119F781E008950A
:1019800084E98093BC0064E080E10C94650C809352
:10199000BB0084E88093BC0063E080E80E94650C93
:1019A0008823A1F08091190481FD0DC08091B900B8
:1019B000887F883241F080911804811106C092E03E
:1019C00090931804089581E0089580E0089510929E
:1019D00018040895809319041092B90088E4809344
:1019E000B8000C94E70CCF93DF93FC0123A52223CE
:1019F00089F0EC010E948F0C811104C080E0DF911E
:101A0000CF9108958EA1811107C00E94C70C882331
:101A1000A9F31BA681E0F3CF80E4F7CF0F931F93C8
:101A2000CF93DF93C62FD42F8901633001F138F4AF
:101A3000613099F0623009F449C0C1E012C06630EB
:101A400029F1673091F16530C1F70E94F30C8111E3
:101A500017C00E94C00CC0E004C0FC0186A50E9413
:101A6000EA0C8C2FDF91CF911F910F910895FC010B
:101A700016A221E023A74111E0CF0E94C00CDDCFC8
:101A80008D2F0E94C70C8111D8CFE3CF0E94F30C99
:101A90008823F9F2DD2389F2F80181918F010E94F8
:101AA000C70C8823B1F2D150F5CF0E94F30C8823E4
:101AB00081F2DD2311F2F80184910E94C70CC82F36
:101AC000882379F20F5F1F4FD150F3CFFC0146A35B
:101AD00021E023A7B2CFDB011496ED91FC9130E019
:101AE00020E065E00994CF92DF92EF92FF920F938E
:101AF0001F93CF93DF938C017B016A0180E0F60195
:101B0000C491811110C081E0CF3F49F04C2FB70143
:101B1000C8010E946B0D882309F44DC080E0BFEF1F
:101B2000CB1ADB0AECCF4FEFCF3F89F3CE3F09F45E
:101B300043C0C03F98F7C03E60F04C2F4F70D701B4
:101B40001496ED91FC9130E020E062E0C801099527
:101B5000E5CFC03D50F04C2F4F70D7011496ED915A
:101B6000FC9130E020E063E0F1CFC03CF8F0D70119
:101B70001496ED91FC9130E020E040E064E0C80173
:101B80000995C295C07FCE5FD0E0CE010E945B0C6C
:101B9000D7011496ED91FC9130E020E041E064E043
:101BA000C8010995CE010E945B0CB8CFC7FDB6CF26
:101BB0008C2F90E0F8CF80E0DF91CF911F910F91B3
:101BC000FF90EF90DF90CF900895AF92BF92CF92A9
:101BD000DF92FF920F931F93CF93DF936C018B01E2
:101BE000F42EE90180E1481709F484C0841758F104
:101BF000AAE04A1709F462C0F80102811381F2E3F6
:101C0000FF1609F4CDC0FF1508F47FC085E1F81672
:101C100009F4CBC0A7E1FA1609F4DCC0B4E1FB1269
:101C20006FC0D8011696ED91FC91179715968C917F
:101C30008E0F9F2F911D11928E179F07E1F7C801FC
:101C40000E94040A5DC0B1E14B1709F45BC0E5E1F5
:101C50004E13D2CFFB01A280B3804FE356E0C60102
:101C60000E94730DD50114964C91406BB801C601CA
:101C70000E946B0DD8011496ED91FC9130E020E0AC
:101C800041E062E0C6010995F50126813781D8015E
:101C90001496ED91FC91D50115964C9166E0C60124
:101CA000099581111CC080E0DF91CF911F910F91A8
:101CB000FF90DF90CF90BF90AF900895DB01149616
:101CC000ED91FC9130E020E042E061E0C601099531
:101CD00047E456E0B801C6010E94730D8DCFD801CC
:101CE0001496ED91FC9130E020E040E063E0C60105
:101CF000099582CF46E356E0B801C6010E94730DF4
:101D000081E0D2CF4BE256E0F7CFE6E4FE1609F4CD
:101D10006BC0F7E4FF1609F46CC08BE3F812F0CF48
:101D200099818B8138E0390F813031F0833011F0A7
:101D3000392F02C0392F985021E0D80113964C91C9
:101D4000491708F420E041E0391708F040E091E03D
:101D5000F8015281351708F490E0322F342B932389
:101D600011F4242369F2FA80D12CC12C843048F478
:101D700090E0FC01E25DFE4FC080865D9E4FDC017D
:101D8000DC90F7FE04C0BE01C8010E94D80988811A
:101D90008C0D888389818D0D8983FF0C91F7B0CFDD
:101DA000BE01C8010E94D809ABCFC8010E94EE094C
:101DB000882309F478CFD8011696ED91FC911797F6
:101DC00015968C918E0F9F2F911D11928E179F0744
:101DD000E1F796CF1882F80182818983858181504D
:101DE0008A8383818B838CCFD80115968C918883CD
:101DF00087CFF8018181FBCFDF92EF92FF920F93A3
:101E00001F93CF93DF93EC01D62E1CAD0BAD7C015D
:101E100084E0E80EF11CE98DFA8DC7010995412F88
:101E2000480F2D2D602FC7010E94480B9BAD890FD5
:101E30008BAF81E090E0DF91CF911F910F91FF90E8
:101E4000EF90DF90089590E080E008958F929F9248
:101E5000AF92BF92CF92DF92EF92FF92CF93DF9338
:101E6000C4EED5E0988121E020936C0490938E0419
:101E700010926D0410928F04682F8DE295E00E94FD
:101E80008D090E94800763E088810E946708109294
:101E90001F0480931E048DE295E00E944609092EDE
:101EA000000CAA0BBB0B8824982EA92EBA2E8DE20B
:101EB00095E00E944609092E000CAA0BBB0B6C0191
:101EC0007D01C828D928EA28FB28FE2CED2CDC2C23
:101ED000CC248DE295E00E944609BC01990F880B45
:101EE000990B6C297D298E299F29DF91CF91FF9035
:101EF000EF90DF90CF90BF90AF909F908F9008951C
:101F00008F929F92AF92BF92CF92DF92EF92FF9209
:101F10000F931F932091ED052F3F19F48AEF0E9434
:101F2000260F0091F1051091F20530E020E0C72E58
:101F3000D82EE92EFF24E7FCFA94C01AD10AE20A4F
:101F4000F30A57E095958795779567955A95D1F758
:101F5000000F111F221F331F4B015C01801A910AD1
:101F6000A20AB30AA5019401A091F305B091F4056A
:101F70000E9466324B015C01FBE0B594A7949794F4
:101F80008794FA95D1F7A7019601C701B6010E947F
:101F9000CE359B01AC01ACE055954795379527951B
:101FA000AA95D1F7A091F505B091F6050E94663289
:101FB0009B01AC01BEE05595479537952795BA959D
:101FC000D1F7280D391D4A1D5B1D2093E90530937B
:101FD000EA054093EB055093EC05A5E0B0E00E94C4
:101FE0005B3260587F4F8F4F9F4F672F782F892F1D
:101FF000992787FD9A950E94063120E030E048EC51
:1020000052E40E9443331F910F91FF90EF90DF90B5
:10201000CF90BF90AF909F908F9008952F923F9256
:102020004F925F926F927F928F929F92AF92BF92E8
:10203000CF92DF92EF92FF920F931F93CF93DF9394
:10204000CDB7DEB76B970FB6F894DEBF0FBECDBF2E
:102050000E94800F8091ED058F3F39F487EF0E9439
:10206000260F6E8B7F8B888F998F8091E9059091D9
:10207000EA05A091EB05B091EC056C017D01FF0C28
:10208000CC08DC2C76019C01AD016C2D7C2D8C2DB7
:102090009C2D345F41405109610971098109910901
:1020A00029873A874B87652E762E872E982E9B8F11
:1020B0005901C42ED52EE62EF72E082F192F0E9477
:1020C000F835322E232E488B598B6A8B7B8B8C8B69
:1020D0009D8B3091FA052091F905932F990F990B5B
:1020E000492F592F692F792F892F0E94F8350CE03D
:1020F0000E94F03629833C874A8F5D876E877F87F1
:10210000582E492E3091FC052091FB05932F990FF5
:10211000990BA32CB22CC888D988EA88FB880C8933
:102120001D89492F592F692F792F892F0E94F83542
:1021300008E00E940937A980BC84CA8CDD84EE8443
:10214000FF84052D142D0E94263770588F4F9F4F06
:10215000E091F705F091F8055F01D12CC12CE12C3D
:10216000F12C8701E983BA82CB82DC82ED82FE8288
:102170000F831887C12CD12CE12CF12C00E010E04A
:102180000E94F83501E20E9409372A8F532E4983B5
:102190005C876D877E878F87492EA0E00E94383745
:1021A00009F436C13091020620910106932F990F50
:1021B000990BA32CB22CC888D988EA88FB880C8993
:1021C0001D89492F592F692F792F892F0E94F835A2
:1021D0001901488B598B6A8B7B8B8C8B9D8B309133
:1021E00000062091FF05932F990F990BA984BA84BB
:1021F000CB84D62CE72CF82C092D1B8D492F592F79
:10220000692F792F892F0E94F83501E10E94F0365D
:102210005101C888D988EA88FB880C891D890E94E9
:10222000263759016A017B01382E192F4E895F89A3
:10223000688D798D84E075956795579547958A9552
:10224000D1F780E090E0A0E1B0E0841B950BA60BF5
:10225000B70B3C014D01990C6608762C43019C019B
:10226000AD01662D762D862D962D0FE10E94F0365C
:10227000722E832E942E5987B62FA72FF82FE92F71
:102280003091FE052091FD05932F990F990B492F51
:10229000592F692F792F892F03E20E94F036032DE1
:1022A0000E94263759016A017B018C01272D382DA8
:1022B000492D59856B2F7A2F8F2F9E2F0E942F37F4
:1022C000E5E3AE2EFCE0BF2EC12CD12CE12CF12C8D
:1022D00000E010E00E94F835AA8CB52CC980DC849F
:1022E000ED84FE840F85142D0E9452362F873E8781
:1022F00049875A876B8779838C879D870DE00E9479
:102300000937922E832E742E652E562E472E382E88
:10231000292E3091080620910706932F990F990BCB
:10232000A92CB82CC72CD62CE52CF42C032D122D5F
:10233000492F592F692F792F892F0E94F8350E9434
:10234000F83509E10E940937AF84BE84C984DA8474
:10235000EB84F9800C851D850E94263719012A011E
:102360003B014C013091060620910506932F990FF1
:10237000990B492F592F692F792F892F0E94F835F2
:1023800003E10E94093759016A017B018C01910127
:10239000A201B301C4010E94263708E00E94093758
:1023A00059016A017B01E82F192F30910406209111
:1023B0000306932F990F990B492F592F692F792FC6
:1023C000892F04E00E94F0360E2F0E9426370E94CB
:1023D000EB3320E030E040E85BE30E9465316B9630
:1023E0000FB6F894DEBF0FBECDBFDF91CF911F9126
:1023F0000F91FF90EF90DF90CF90BF90AF909F90A4
:102400008F907F906F905F904F903F902F900895A6
:1024100060E070E0CB01E3CFCF939091ED059F3F5B
:1024200041F5682F8091E40591E090936C048093CE
:102430008E0410926D0410928F048DE295E00E943C
:102440008D090E94800762E08091E4050E94670880
:1024500010921F0480931E048DE295E00E944609AD
:10246000C82F8DE295E00E94460920E03C2F282BE2
:10247000392B922F832FCF9108950F931F93CF93D2
:10248000DF93FC01048115810115110539F4FB016D
:102490001082DF91CF911F910F9108954150510902
:1024A0004017510708F48A01EB01FC01608171813A
:1024B000A801CE010E944C39C00FD11F1882E9CF6C
:1024C000CF93DF93C091D805D091D905209761F0C3
:1024D0008991882349F0082E000C990B0E94263917
:1024E000FE0131978083F4CFDF91CF91089585ED80
:1024F0008093BC008091680490916904A0916A0463
:10250000B0916B040796A11DB11D23E0B695A79568
:10251000979587952A95D1F72091BC0024FD03C09B
:102520001092660408954091680450916904609186
:102530006A0470916B04452B462B472B69F3009777
:10254000A105B10541F025E32A95F1F700000197B7
:10255000A109B109E1CF809167040C945F07FC01E8
:1025600080819181009711F00C94A52C60E070E0BF
:10257000CB010895FB0144815581FC012481358103
:102580002417350778F080819181009759F0FB017D
:10259000608171816115710529F00E943E3921E049
:1025A000892B09F020E0822F08950F931F93CF937A
:1025B000DF938C01EB01FC01808191810097E1F0B8
:1025C0006881798161157105A9F0428153812C815F
:1025D0003D814217530770F00E9437398C819D81ED
:1025E000F801958384831D821C82DF91CF911F9116
:1025F0000F9108950E94E03788819981F8019183B5
:1026000080838A819B81938382838C819D81958342
:102610008483198218821B821A82E5CFCF93DF93BD
:10262000EC0188819981009711F00E94E0371982AE
:1026300018821D821C821B821A82DF91CF9108951D
:10264000FC0180819181009711F00C94E03708958E
:102650000F931F93CF93DF93EC01888199810097AB
:1026600059F02A813B812617370730F081E0DF914E
:10267000CF911F910F9108958B016F5F7F4F0E9443
:102680006938009759F0998388831B830A832C81CA
:102690003D81232B59F7FC011082E8CF80E0E7CF82
:1026A000EF92FF920F931F93CF93DF936115710504
:1026B00041F480E0DF91CF911F910F91FF90EF9057
:1026C000089541155105B1F07B01EC010C811D818C
:1026D000040F151FB8010E942813882351F3288185
:1026E00039818C819D81B701820F931F0E943739F8
:1026F0001D830C8381E0DECF0F931F93CF93DF9375
:1027000000D0CDB7DEB78C0119821A8241E050E0CB
:10271000BE016F5F7F4F0E945013811103C0C8013B
:102720000E940E13C8010F900F90DF91CF911F915F
:102730000F910895CF93DF93EC01FB0101900020EE
:10274000E9F73197AF01461B570B0E9450138111D7
:1027500003C0CE010E940E13CE01DF91CF910895E8
:10276000CF93DF93EC01FB0144815581608171813E
:102770000E945013811103C0CE010E940E13CE019E
:10278000DF91CF910895FB01448155816081718172
:102790000C945013EF92FF920F931F93CF93DF93FC
:1027A000EC018B01CB010E94D32C7C01BC01CE013A
:1027B0000E94281381110BC0CE010E940E13CE017E
:1027C000DF91CF911F910F91FF90EF900895FD82BF
:1027D000EC82B801888199810E94CC2CF0CFEF92D5
:1027E000FF920F931F93CF93DF93EC017B018A013C
:1027F000BA010E94281381110BC0CE010E940E1352
:10280000CE01DF91CF911F910F91FF90EF9008952E
:102810001D830C83B701888199810E943739F0CFDD
:10282000FB0101900020E9F73197AF01461B570BE0
:102830000C94EF130F931F93CF93DF93CDB7DEB7B5
:1028400062970FB6F894DEBF0FBECDBF8C01CB01EF
:10285000F8011182108213821282158214824AE0DA
:10286000BE016F5F7F4F0E94DC2CBE016F5F7F4F08
:10287000C8010E94101462960FB6F894DEBF0FBE16
:10288000CDBFDF91CF911F910F910895CF93DF932B
:10289000EC01FB018617970749F060817181611592
:1028A000710541F0448155810E94EF13CE01DF9103
:1028B000CF9108950E940E13F9CFFC01118210826E
:1028C00013821282158214820C944614FC01118228
:1028D000108213821282158214826115710551F0E3
:1028E000FB0101900020E9F73197AF01461B570B20
:1028F0000C94EF130895AF92BF92CF92DF92EF92B4
:10290000FF920F931F93CF93DF936C015B017A01CA
:1029100089012417350720F48F2D7901042F182FF2
:1029200064E671E0C6010E946614D5011496CD914B
:10293000DC91EC16FD06E0F40C171D0708F4E80125
:10294000D501ED91FC911197EC0FFD1F10811082C4
:102950006D917C916E0D7F1DC60161157105A1F011
:102960000E941014F50180819181C80FD91F18832E
:10297000C601DF91CF911F910F91FF90EF90DF90F3
:10298000CF90BF90AF9008950E940E13EBCFCF93DE
:10299000DF93EC01FB01248135810E947B14CE0181
:1029A000DF91CF9108950F931F93CF93DF93CDB70E
:1029B000DEB72C970FB6F894DEBF0FBECDBFFC017B
:1029C000248135811216130664F48C0125313105FA
:1029D0009CF40E94030464E170E080E090E00E94B7
:1029E000E8052C960FB6F894DEBF0FBECDBFDF9181
:1029F000CF911F910F9108952FE030E050E040E01B
:102A0000BC01CE0107960E947B144B855C856F81CB
:102A1000788580E994E00E94D60369E170E080E067
:102A200090E00E94E8054FE050E0B801CE01019629
:102A30000E94C714BE016F5F7F4FCE0107960E94B0
:102A4000D512CE0101960E942013CE0107960E9456
:102A5000030464E170E080E090E00E94E80564E631
:102A600071E0CE0107960E941014CE0107960E94D5
:102A70002013B7CFEF92FF920F931F93CF93DF9363
:102A8000CDB7DEB7A1970FB6F894DEBF0FBECDBFAE
:102A90007C01CB01BA01F7011182108213821282EC
:102AA0001582148242E0420F8E010F5F1F4F0E9479
:102AB000832C009789F0BC01C7010E941014A196D5
:102AC0000FB6F894DEBF0FBECDBFDF91CF911F913F
:102AD0000F91FF90EF900895C7010E940E13EFCF62
:102AE0000F931F93CF93DF93D62FC42F10926601BD
:102AF00010926501FC01448155814F5F5F4F21F0C9
:102B000065E671E00E943D12E0913906F0913A06C7
:102B100084E296E00995C80F05E611E0F8012191DD
:102B20008F01211105C0DF91CF911F910F91089561
:102B30004C2F6D2F84E296E00E94480BD80FEECF09
:102B40008F929F92AF92BF92CF92DF92FF920F939C
:102B50001F93CF93DF93CDB7DEB7AE970FB6F89440
:102B6000DEBF0FBECDBF6C015B018A010E94F7067C
:102B70001CA21BA21EA21DA218A61FA228EE33E0B3
:102B800040E050E00E943C32CA01B90120E831E542
:102B900041E050E00E943C322AE0AE014F5F5F4FBF
:102BA0000E94E72CBE016F5F7F4FCE0183960E948B
:102BB0001014BE016D5D7F4FCE0101960E945D1421
:102BC00063EA72E0CE0101960E949A13BC01CE0125
:102BD00089960E945D14CE0101960E942013CE01B9
:102BE00083960E94201380912806909129068F5188
:102BF000924071F08FE192E090932906809328062D
:102C00000E94950383E993E090933A0680933906F6
:102C100010923B060E9495038DE19BE090933A064B
:102C20008093390680912F06803309F0B3C08FEF6F
:102C3000809344068093450680915D06811105C00E
:102C400081E080935D060E94F10A809026069090B4
:102C50002706E0915506F091560682E00995E0912D
:102C60005506F091560681E0099530E020E044E1F8
:102C7000B40184E296E00E940B0A27E536E047E1C2
:102C8000B40184E296E00E940B0AE0915506F091AF
:102C9000560680E00995BE01675D7F4FCE01019623
:102CA0000E945D1441E060E0CE0101960E94701523
:102CB000CE0101960E942013B601CE0101960E941A
:102CC0005D1441E062E3CE0101960E947015CE01D1
:102CD00001960E942013B501CE0101960E945D1459
:102CE00040E160E0CE0101960E947015CE01019690
:102CF0000E942013E0913206F0913306309719F0CC
:102D000084E296E009958090260690902706E0914F
:102D10005506F091560682E00995E0915506F0912E
:102D2000560681E0099530E020E045E1B40184E2F7
:102D300096E00E940B0AF82E882341F027E536E042
:102D400047E1B40184E296E00E940B0AE091550647
:102D5000F091560680E00995F1109DCFB801110F52
:102D6000880B990B0E94E805CE0189960E942013DA
:102D7000AE960FB6F894DEBF0FBECDBFDF91CF91F8
:102D80001F910F91FF90DF90CF90BF90AF909F90D9
:102D90008F900895883231F0823031F081E0809355
:102DA00044064ACF8FEFFBCF83E0F9CFFF920F931A
:102DB0001F93CF93DF93EC01F62E08811981C80190
:102DC0000E942632F81621F06F2DC8010E942E3283
:102DD000CE01DF91CF911F910F91FF900895EF9257
:102DE000FF920F931F93CF93DF9300D0CDB7DEB741
:102DF00009E315E0895395407C01C701800F911FBD
:102E00009A838983F80161918F01CE0101960E9416
:102E1000D616F5E007381F0781F789E395E00F9094
:102E20000F90DF91CF911F910F91FF90EF90089538
:102E3000EF92FF920F931F93CF93DF9300D0CDB704
:102E4000DEB70DE815E08D5895407C01C701800F75
:102E5000911F9A838983F80161918F01CE010196B8
:102E60000E94D616F5E0043B1F0781F78DE895E038
:102E70000F900F90DF91CF911F910F91FF90EF90E6
:102E800008952F923F924F925F926F927F928F920E
:102E90009F92AF92BF92CF92DF92EF92FF920F93E9
:102EA0001F93CF93DF93CDB7DEB76E970FB6F8942D
:102EB000DEBF0FBECDBF1A8219821C821B821E820A
:102EC0001D8267E276E0CE0101960E94CA13BE0120
:102ED0006F5F7F4F88ED95E00E94BA12182FCE01E8
:102EE00001960E942013112311F164E771E0CE01D5
:102EF00001960E94661464EB75E0CE0101960E9473
:102F0000B013BC018EED95E00E944614CE010196EF
:102F10000E9420136EED75E0CE0101960E945D14B3
:102F2000CE0101960E94D314CE01019600C41A82EC
:102F300019821C821B821E821D8263E276E0CE0112
:102F400001960E94CA13BE016F5F7F4F88ED95E026
:102F50000E94BA12182FCE0101960E94201311234D
:102F600069F06EE771E08EED95E00E9410146AEB57
:102F700075E08EED95E00E94C313CCCF6CE871E054
:102F8000CE0101960E946614BE016F5F7F4F88EDEF
:102F900095E00E94BA12182FCE0101960E942013CC
:102FA0001123D9F127E030E046E050E06CEC75E009
:102FB000CE0101960E947B14BE016F5F7F4F86ECAD
:102FC00095E00E94D512CE0101960E94201386EC56
:102FD00095E00E94AF12672B21F410920E0481E05D
:102FE00003C081E080930E046E960FB6F894DEBFA6
:102FF0000FBECDBFDF91CF911F910F91FF90EF904A
:10300000DF90CF90BF90AF909F908F907F906F9008
:103010005F904F903F902F90089563E971E0CE014B
:1030200001960E946614BE016F5F7F4F88ED95E0A8
:103030000E94BA12182FCE0101960E94201311236C
:1030400009F4BAC08091BD039091BE031816190609
:1030500034F688EC90E090930D0180930C0180E9A8
:1030600094E00E94DC041D861E861F86188ACC24EC
:10307000C394D12C40EC242E43E0342E5E012DE08D
:10308000A20EB11C2E0131E1430E511C5DEB652EE9
:1030900053E0752E8091BD039091BE038C159D0564
:1030A0000CF49DCF80910C0190910D01813C9340D7
:1030B00024F030920D0120920C0100910C0110912E
:1030C0000D01750148018A189B08C4018E0D9F1DD2
:1030D0000E942632F70181937F01E415F505A9F7D7
:1030E000C801049690930D0180930C0129E9E22E0A
:1030F00023E0F22E05591340C8018E0D9F1D0E943A
:103100002632F70181937F016E167F06A9F74D8560
:103110005E856F85788923E0CE0107960E943A1577
:10312000BE01695F7F4FCE0101960E945D1467E981
:1031300071E0CE0101960E949A13BC018EED95E0DC
:103140000E944614CE0101960E942013CE010796DC
:103150000E94201369E973E0CE0101960E94661473
:10316000BE016F5F7F4F8EED95E00E94C313CE01CD
:1031700001960E9420136EED75E0CE0101960E942B
:103180005D14CE0101960E94D314CE0101960E94D7
:10319000201380910C0190910D01849690930D0164
:1031A00080930C0164E170E080E090E00E94E8050B
:1031B000FFEFCF1ADF0A6ECF6AE971E0CE01019608
:1031C0000E946614BE016F5F7F4F88ED95E00E94FC
:1031D000BA12182FCE0101960E9420131123F1F18B
:1031E00026E030E045E050E06CEC75E0CE01019661
:1031F0000E947B14BE016F5F7F4F86EC95E00E94BA
:10320000D512CE0101960E94201386EC95E00E9413
:10321000AF12672B19F410929803E1CE81E08093EE
:10322000980388EC90E090930D0180930C0110922C
:10323000BE031092BD031092940310929503109256
:103240009603109297030E94F70660939003709381
:1032500091038093920390939303C1CE60EA71E04F
:10326000CE0101960E946614BE016F5F7F4F88ED0C
:1032700095E00E94BA12182FCE0101960E942013E9
:10328000112309F479C08091D0059091D105079759
:1032900008F4A5CE46E050E06CEC75E0CE01019656
:1032A0000E94C714BE016F5F7F4F86EC95E00E94BD
:1032B000D512CE0101960E9420138091C6059091EF
:1032C000C705C12CD12C7601009721F00E94A12CBA
:1032D0006B017C01C0921A01D0921B01E0921C018B
:1032E000F0921D0167EA71E08EED95E00E941014E6
:1032F00022E0B701A601CE0107960E943A15BE0151
:10330000695F7F4FCE0101960E945D1463EA72E00F
:10331000CE0101960E949A13BC018EED95E00E94A9
:10332000C313CE0101960E942013CE0107960E947E
:1033300020136EED75E0CE0101960E945D14CE0162
:1033400001960E94D314CE0101960E9420130E9480
:10335000F70628EE33E040E050E00E94A532CA01B3
:10336000B9010E9404316093130470931404809394
:1033700015049093160433CE62EB71E0CE010196F2
:103380000E946614BE016F5F7F4F88ED95E00E943A
:10339000BA12182FCE0101960E942013112309F4AE
:1033A00057C08091D0059091D105079708F417CEAA
:1033B00046E050E06CEC75E0CE0101960E94C71427
:1033C000BE016F5F7F4F86EC95E00E94D512CE0163
:1033D00001960E9420138091C6059091C705C12CCB
:1033E000D12C7601009721F00E94A12C6B017C0169
:1033F000C0920801D0920901E0920A01F0920B01FB
:1034000069EB71E08EED95E00E94101421E0B701A8
:10341000A601CE0107960E943A15BE01695F7F4F53
:10342000CE0101960E945D1463EA72E0CE0101961E
:103430000E949A13BC018EED95E00E94C313CE0149
:1034400001960E942013CE0107960E94201362CDA0
:1034500064EC71E0CE0101960E946614BE016F5FBC
:103460007F4F88ED95E00E94BA12182FCE01019689
:103470000E942013112341F126E030E044E050E0A7
:103480006CEC75E0CE0101960E947B14BE016F5F6B
:103490007F4F86EC95E00E94D512CE0101960E94E6
:1034A000201386EC95E00E94AF1270933A0560936A
:1034B000390570931701609316018091180190915E
:1034C00019010E94EF168BCD69EC71E0CE010196D7
:1034D0000E946614BE016F5F7F4F88ED95E00E94E9
:1034E000BA12182FCE0101960E9420131123A9F1C0
:1034F00043E050E06CEC75E0CE0101960E94C714E9
:10350000BE016F5F7F4F86EC95E00E94D512CE0121
:1035100001960E94201366EC75E0CE0101960E9490
:103520005D14CE0101960E947C13BC018AEB95E0EC
:103530000E944614CE0101960E9420134091BE05C0
:103540005091BF054115510509F4B7CF6BE375E004
:103550008AEB95E00E943D12B0CF60ED71E0CE01A4
:1035600001960E946614BE016F5F7F4F88ED95E063
:103570000E94BA12182FCE0101960E942013112327
:1035800009F489C08091D0059091D105409708F049
:1035900022C342E050E06CEC75E0CE0101960E943F
:1035A000C714BE016F5F7F4F86EC95E00E94D51275
:1035B000CE0101960E9420138091C6059091C70507
:1035C000009709F441C00E94A12C20E030E048ECB3
:1035D00052E40E9465310E94B533609345057093B3
:1035E000460580934705909348056DEC71E08EED9C
:1035F00095E00E94101460914505709146058091F8
:103600004705909148058B019C0100591F452140B9
:10361000310901341C4921053105D0F066EC75E013
:10362000CE0101960E945D1463ED71E0CE0101961A
:103630000E949A13BC018EED95E00E94C313CE0147
:1036400001960E942013CBCC60E070E0CB01BDCF8F
:103650000E94063120E030E048EC52E40E944333FF
:10366000AB01BC0122E0CE0101960E943A15BE01D9
:103670006F5F7F4F8EED95E00E94C313CE010196E0
:103680000E94201343E050E060EE71E08EED95E083
:103690000E94501312CF64EE71E0CE0101960E9499
:1036A0006614BE016F5F7F4F88ED95E00E94BA12ED
:1036B000182FCE0101960E9420131123D9F1809179
:1036C000850590918605019709F089CC64E671E043
:1036D000CE010D960E94661489899A89009729F176
:1036E000ED85FE852081222301F10797F0F06AEE37
:1036F00071E0CE0107960E946614BE01635F7F4FA2
:10370000CE0107960E94B013BC01CE0101960E9423
:103710005D14CE0101960E94D314CE0101960E9441
:103720002013CE0107960E942013CE010D960E9411
:10373000201355CC6FEE71E0CE0101960E94661405
:10374000BE016F5F7F4F88ED95E00E94BA12182F7F
:10375000CE0101960E9420131123F1F025E030E004
:1037600044E050E06CEC75E0CE0101960E947B14C1
:10377000BE016F5F7F4F86EC95E00E94D512CE01AF
:1037800001960E94201386EC95E00E94AF12709380
:1037900086056093850591CE64EF71E0CE010196B8
:1037A0000E946614BE016F5F7F4F88ED95E00E9416
:1037B000BA12182FCE0101960E942013112309F48A
:1037C0005EC009E110E0C12CD12C760180E10E949D
:1037D000A805BC01990F880B990B0E9406319B012B
:1037E000AC01C701B6010E94D7326B017C016AE0CF
:1037F00070E080E090E00E94E8050150110931F787
:1038000020E030E040EA50E4C701B6010E94653193
:1038100020E030EC4FE754E40E94433320E030E0F6
:1038200048EC51E40E944333609361057093620554
:10383000809363059093640580911801909119011C
:103840000E94EF1668EF71E08EED95E00E94101473
:103850004091610550916205609163057091640526
:1038600022E0CE0107960E943A15BE01695F7F4FA4
:10387000CE0101960E945D1460E072E0D7CD63E056
:1038800072E0CE0101960E946614BE016F5F7F4F09
:1038900088ED95E00E94BA12182FCE0101960E9481
:1038A0002013112309F49BCB43E050E068ED75E051
:1038B000CE0107960E94C714BE01695F7F4FCE01FB
:1038C00001960E945D14CE0101960E947C13BC01FA
:1038D00086EC95E00E944614CE0101960E942013CA
:1038E000CE0107960E94201366EC75E0CE01499642
:1038F0000E945D1467E072E0CE0101960E9466149A
:103900008D8D9E8D892BC9F1098D1A8D69817A81E2
:10391000C8010E945B39009781F1FC01E01BF10BAB
:103920008F01CE0101960E94201364E671E0CE0162
:1039300043960E94661464E671E0CE010D960E94E3
:10394000661410161106E4F469E072E0CE010196E7
:103950000E946614CE0101960E94D314CE010196F6
:103960000E942013CE010D960E942013CE01439693
:103970000E942013CE014996DACE0FEF1FEFD1CF70
:10398000BE01675E7F4FCE010D960E944614D12C7A
:10399000C12C8AEF682E77247A9496E0592E898973
:1039A0009A89009709F408C1F5E0CF16D104C9F34C
:1039B00068EE71E0CE0101960E946614BE016F5F51
:1039C0007F4FCE010D960E94BA12182FCE0101969C
:1039D0000E9420131111C9C001E010E0980150E0CD
:1039E00040E0BE01635F7F4FCE0107960E947B14CB
:1039F000BE01695F7F4FCE0101960E945D14CE012A
:103A000001960E947C13BC01CE0143960E9446148D
:103A1000CE0101960E942013CE0107960E9420132A
:103A2000BE016D5E7F4FCE0107960E945D148B85AF
:103A30009C85029708F49CC068EE71E0CE01019667
:103A40000E946614BE016F5F7F4FCE0107960E94F1
:103A5000BA12F82ECE0101960E942013FF2009F41D
:103A600087C022E030E041E050E0BE01695F7F4F57
:103A7000CE0101960E947B14CE0101960E94AF12E6
:103A80004B017B01CE0101960E94201397FE03C0DB
:103A90002CE1E20EF11CB3016E197F095C9C7001F0
:103AA0005D9CF00C1124F701E357FA4F7687658788
:103AB000CE0107960E942013B7016A567A4F44E060
:103AC00050E0CE0143960E943D123FEFC31AD30A45
:103AD00089899A890817190708F067C0A801BE01EB
:103AE000635F7F4FCE0101960E94C714BE016F5FD6
:103AF0007F4FCE0143960E94D512CE0101960E94BF
:103B00002013BE016D5E7F4FCE010D960E944614BC
:103B1000AD84BE84A114B10409F441CF09891A8986
:103B200075010115110509F43ACF47014FEF841AC9
:103B3000940AF7018081082E000C990B0E94CE3068
:103B4000892BD9F4015011090A0D1B1DF801808140
:103B5000082E000C990B0E94CE30892B81F00E1597
:103B60001F0568F001501109F1CF02E010E036CFD7
:103B7000CE0107960E94AF1291CF7401D6CF0F5F8E
:103B80001F4FA8014E195F095A8B498BAE14BF0411
:103B900020F4B701C5010E942E39ED85FE85898983
:103BA0009A89E80FF91F1082FACE64E671E0CE011F
:103BB0000D960E941014F3CEC0928F05CC2041F0D8
:103BC00081E080938D058EE190E00E941817CACEA7
:103BD00010928D05F8CF80E007CA2F923F924F9246
:103BE0005F926F927F928F929F92AF92BF92CF928D
:103BF000DF92EF92FF920F931F93CF93DF93CDB796
:103C0000DEB7A3970FB6F894DEBF0FBECDBF7C0121
:103C100064E671E08EED95E00E941014C7010596F0
:103C2000059768F080911704811109C02CEEE21607
:103C30002FEFF20624F0F0921204E0921104F70143
:103C40007A96E432F10508F0D9C6E75DF14E0C949E
:103C5000F2358B24FE248724FE24FE24FE24FE2439
:103C6000FE24FE24FE24FE24481F481F481F481F30
:103C70004D1E481F481F3120481F481F3420432035
:103C80004620FE24481F481F54207522AD235F2480
:103C90007D24481F481F481F481F60E080E10E94A4
:103CA0007705809117048111D7C18AE090E0A0E0E8
:103CB000B0E088A399A3AAA3BBA360E272E08EED53
:103CC00095E00E941014312C212C1E8E1F8EC12CC9
:103CD000D12C760102E310E0812C912C540180E17B
:103CE0000E94A805092E000CAA0BBB0B880E991E7A
:103CF000AA1EBB1E65E070E080E090E00E94E8052F
:103D00000150110961F74090610550906205609083
:103D1000630570906405C501B4010E94063120E07E
:103D200030E040EA50E40E94653120E030E040E8B5
:103D30005AE30E94653120E030E048E452E40E94FA
:103D40004333A30192010E94D63220E030E040E7E5
:103D500051E40E9465314B015C01A30192016AE9C3
:103D600079E989E390E40E94D6329B01AC01C50158
:103D7000B4010E94433320E030E0A9010E94D73211
:103D800020E030E040E251E40E9465315B018C01AB
:103D9000232D322D4E8D5F8D0E943F34181624F452
:103DA0003A2C2B2C0E8F1F8F9FEFC91AD90AE90AC4
:103DB000F90A88A199A1AAA1BBA18C159D05AE0500
:103DC000BF050CF087CF6EE170E080E090E00E94CC
:103DD000E80567E272E08EED95E00E94101422E0A3
:103DE000432D522D6E8D7F8DCE0101960E943A1586
:103DF000BE016F5F7F4FCE0142960E945D1464E367
:103E000072E0CE0142960E949A13BC0186EC95E0C6
:103E10000E944614CE0142960E942013CE010196C4
:103E20000E9420136EED75E0CE0142960E945D1453
:103E300066EC75E0CE0101960E945D1444E650E008
:103E4000BE016E5E7F4FCE0101960E94A015CE018D
:103E500001960E942013CE0142960E9420136BE32C
:103E600072E0CE0101960E94661466EC75E0CE0108
:103E700001960E94B0136EED75E00E94B013BC0174
:103E80008EED95E00E944614CE0101960E9420130B
:103E90008091E2059091E305892B09F4BEC06EED97
:103EA00075E0CE0101960E945D14CE0101960E943C
:103EB000D314CE0101960E9420136EED75E0CE0161
:103EC00042960E945D1480919803882309F4A1C052
:103ED0008091BD039091BE03843191050CF099C08F
:103EE00000910C0110910D01013CF3E01F070CF053
:103EF00090C001969093BE038093BD030E94F70685
:103F0000C0909003D0909103E0909203F0909303BF
:103F10006C197D098E099F090E94043120E030E070
:103F20004AE754E40E9443336093940370939503EB
:103F30008093960390939703083C110534F488EC22
:103F400090E090930D0180930C0180910C01909171
:103F50000D0104E913E09C01245933407901C701A4
:103F6000800F911F9A838983D8016D918D01CE01B5
:103F700001960E94D616B3E008391B0781F7E0903E
:103F80000C01F0900D01C701049690930D018093F0
:103F90000C01BE016E5E7F4FCE0101960E945D1442
:103FA000CE0101960E947C13BC018EED95E00E942B
:103FB0004614CE0101960E9420134091E2055091D3
:103FC000E3054115510531F069E973E08EED95E0A7
:103FD0000E943D1209E913E0F701E559F3407F0122
:103FE000C701800F911F9A838983D8016D918D013C
:103FF000CE0101960E94D616B3E00D3B1B0781F758
:1040000080910C0190910D01849690930D01809305
:104010000C01CE0142960E94201364E670E080E01D
:1040200090E00E94E805A3960FB6F894DEBF0FBE9D
:10403000CDBFDF91CF911F910F91FF90EF90DF9057
:10404000CF90BF90AF909F908F907F906F905F9038
:104050004F903F902F90089583E090E0A0E0B0E073
:1040600028CE0E94F70614CF80911704882321F0F0
:104070008EED95E00E94030468EC70E080E090E033
:104080000E94E80505CF1092170402CF81E08093CB
:1040900017048093950580911104909112049093D8
:1040A000100480930F04F4CE64E670E080E090E0AA
:1040B0000E94E80580911601909117010B9731F548
:1040C00080911F06882309F0F89482E10E9474060B
:1040D0008C0180911F06882309F078940115110541
:1040E00009F457C180E090ECA9E7B4EC8093120684
:1040F00090931306A0931406B093150680931606AA
:1041000090931706A0931806B09319068091160194
:1041100090911701469731F580911F06882309F089
:10412000F89481E00E9474068C0180911F06882318
:1041300009F078940115110509F48CC180E090EC28
:10414000A9E7B4EC8093120690931306A09314068B
:10415000B09315068093160690931706A093180641
:10416000B093190664E670E080E090E00E94E805F4
:10417000012B09F08DCE8091160690911706A09123
:104180001806B091190680938C0390938D03A09329
:104190008E03B0938F038091120690911306A09125
:1041A0001406B09115068093880390938903A09319
:1041B0008A03B0938B0364E671E0CE0148960E94B7
:1041C000661440911606509117066091180670917A
:1041D000190620E0CE0101960E943A15BE016F5FDC
:1041E0007F4FCE0148960E94D512CE0101960E94C3
:1041F0002013BE01685E7F4FCE0101960E945D14C0
:104200006FE372E0CE0101960E949A13BC018EED1D
:1042100095E00E944614CE0101960E942013409121
:10422000120650911306609114067091150620E055
:10423000CE0101960E943A15BE016F5F7F4FCE01FD
:1042400048960E94D512CE0101960E942013BE010D
:10425000685E7F4FCE0101960E945D1463E472E0B8
:10426000CE0101960E949A13BC018EED95E00E944A
:10427000C313CE0101960E94201365E472E0CE01C3
:1042800042960E9466146EED75E0CE0101960E9482
:104290005D1444E650E0BE016E5E7F4FCE01019694
:1042A0000E94A015CE0101960E942013CE014296D5
:1042B0000E94201340918C0350918D0360918E03D6
:1042C00070918F0321E0CE0101960E943A15BE0144
:1042D0006F5F7F4FCE0148960E94D512CE010196A6
:1042E0000E9420136AEC71E0CE0101960E946614D0
:1042F000BE01685E7F4FCE0101960E94B0136FE34E
:1043000072E00E949A13BC018EED95E00E94461463
:10431000CE0101960E942013409188035091890399
:1043200060918A0370918B0321E0CE0101960E9477
:104330003A15BE016F5F7F4FCE0148960E94D5129D
:10434000CE0101960E94201363E572E0CE01019632
:104350000E946614BE01685E7F4FCE0101960E94E6
:10436000B01363E472E00E949A13BC018EED95E0F5
:104370000E94C313CE0101960E94201364E670E0F0
:1043800080E090E00E94E805CE0148960E9420134C
:104390007FCD10911A06E0901B066E2D70E090E024
:1043A00080E00E9406312DEC3CEC4CEC5DE30E9479
:1043B00065314B015C01612F70E090E080E00E946C
:1043C00006319B01AC01C501B4010E94D732609354
:1043D00012067093130680931406909315060091AD
:1043E0001C06F0901D06602F6F7770E090E080E073
:1043F0000E9406314B015C016F2D70E090E080E07F
:104400000E9406312DEC3CEC4CEC5DE30E946531E2
:104410009B01AC01C501B4010E94D73207FD18C051
:1044200060931606709317068093180690931906EA
:104430001E0D100F1F0D81E090E020911E0612133B
:1044400002C090E080E000271127081B190B5ECE08
:104450009058E6CF10911B0600911A0660911A063B
:1044600070911B0676276727762790E080E00E94F0
:1044700004312DEC3CEC4CEC5DE30E946531609323
:104480001206709313068093140690931506E0901D
:104490001D06F0901C066F2D6F77762F6E2D90E025
:1044A00080E00E9404312DEC3CEC4CEC5DE30E947A
:1044B0006531F7FC18C06093160670931706809359
:1044C000180690931906100F1E0D1F0D81E090E045
:1044D00020911E06121302C090E080E000271127F1
:1044E000081B190B3FCE9058E6CF80911501882309
:1044F00009F4CECC0E940E102B013C010E94800FCB
:104500004B015C016091450570914605809147051E
:10451000909148050E94063120E030E048EC52E4DA
:104520000E9443336B017C010E940E1020E030E0BA
:1045300048EC52E40E944333A70196010E944333A2
:1045400021E03EED42E45EE30E9444349B01AC0175
:1045500060E070E080E89FE30E94D63220E03AE21B
:104560004DE257E40E9465316B017C0120E030E0B0
:1045700048EC52E4C301B2010E944333AB01BC01D9
:1045800022E0CE0142960E943A15BE016E5E7F4F38
:10459000CE0101960E945D1466E572E0CE0101969F
:1045A0000E949A13BC0180EC95E00E944614CE0153
:1045B00001960E942013CE0142960E94201360ECC7
:1045C00075E086EC95E00E94461460ED71E0CE0146
:1045D00001960E94661460EC75E0CE0101960E947F
:1045E000B013BC0180EC95E00E944614CE01019608
:1045F0000E94201321E0B501A401CE0142960E9441
:104600003A15BE016E5E7F4FCE0101960E945D1489
:104610006BE572E0CE0101960E949A13BC018EED0B
:1046200095E00E944614CE0101960E942013CE010F
:1046300042960E94201320E0B701A601CE014296C7
:104640000E943A15BE016E5E7F4FCE0101960E9418
:104650005D146EE572E0CE0101960E949A13BC01D2
:1046600086EC95E00E94C313CE0101960E942013B0
:10467000CE0142960E94201366EC75E0CE010196B1
:104680000E945D146EED75E0CE0142960E945D14AD
:1046900044E650E0BE016F5F7F4FCE0142960E941C
:1046A000A015CE0142960E942013CE0101960E94D1
:1046B00020136AEC71E0CE0101960E9466146EED43
:1046C00075E0CE0101960E94B01360E672E00E9490
:1046D0009A13BC018EED95E00E944614CE0101961E
:1046E0000E94201321E0B701A601CE0142960E944C
:1046F0003A15BE016E5E7F4FCE0101960E945D1499
:104700006EE572E0CE0101960E949A13BC018EED17
:1047100095E00E94C313CE0101960E942013CE01A2
:1047200042960E94201360EC75E0CE0101960E9433
:104730005D146EED75E0CE0101960E94B013BC01D0
:104740008EED95E00E944614CE0101960E94201342
:1047500065E070E080E090E093CC8BE0E82EF12CF7
:1047600010E000E09924939493E2892E90926C04D7
:1047700080928E0410926D0410928F0462E083E2A6
:104780000E94670810921F0480931E048DE295E03A
:104790000E944609D82EC12C8DE295E00E94460960
:1047A0005C01AC28BD280E948007B50190E080E044
:1047B0000E9404312AE939E949E95FE30E94433361
:1047C0000E94BC330617170708F48B0162E370E000
:1047D00080E090E00E94E80591E0E91AF10831F6E6
:1047E00064E672E08EED95E00E9410141B8A1A8A2E
:1047F0001D8A1C8A1F8A1E8A4AE0BE016F5F7F4F96
:10480000C8010E942D2DBE016F5F7F4FCE014296E1
:104810000E941014BE016E5E7F4FCE0101960E9471
:104820005D1464E772E0CE0101960E949A13BC0108
:1048300086EC95E00E944614CE0101960E9420135A
:10484000CE0142960E9420136EED75E0CE010196D6
:104850000E945D1466EC75E0CE0142960E945D14E4
:1048600044E650E0BE016F5F7F4FCE0142960E944A
:10487000A015CE0142960E942013CE0101960E94FF
:10488000201369E772E0CE0101960E94661466EC7F
:1048900075E0CE0101960E94B0136EED75E00E94A6
:1048A000B013BC018EED95E00E944614CE01019636
:1048B0000E94201362E370E080E090E0E1CB81E0B1
:1048C00080930E010E941B068C016CE772E08EED56
:1048D00095E00E94101460E074E0601B710BCE0143
:1048E00001960E941A14BE016F5F7F4F8EED95E016
:1048F0000E94C313CE01019649CD6CE872E08EEDA3
:1049000095E00E9410140E941B06BC01E8CFF0E065
:10491000E0E00995BDCA80918F0518160CF055C0CE
:1049200081E080938D0567E972E08EED95E00E944D
:10493000101480918D05882309F44AC065EA72E05D
:10494000CE0101960E9466146EED75E0CE010196CF
:104950000E94B013BC018EED95E00E944614CE017A
:1049600001960E9420136EED75E0CE0101960E9423
:104970005D14CE0101960E94D314CE0101960E94CF
:10498000201368EE73E080E090E00E94E8058091DB
:104990008D0581110E94052564E671E08EED95E09C
:1049A0000E9410148091170480939505811170CA9C
:1049B00067EE71E082ED95E00E94101486EE9FEFA5
:1049C000909312048093110463CA10928D05ABCFAB
:1049D0006DEA72E0CE0101960E9466146EED75E0FC
:1049E000CE0101960E94B013BC018EED95E00E94AD
:1049F0004614CE0101960E942013D4CF66EB72E0DC
:104A00008EED95E00E94101443CA0F931F93CF932D
:104A1000DF930DE815E0D0E0C0E00A5F1F4F809102
:104A20008F05082E000C990BC817D9076CF4F801F4
:104A3000878190850E94ED1D68EE73E080E090E034
:104A40000E94E8052196E9CFDF91CF911F910F9148
:104A500008951F920F920FB60F9211242F933F9338
:104A60004F935F936F937F938F939F93AF93BF9376
:104A7000EF93FF9380E994E00E946D04FF91EF9122
:104A8000BF91AF919F918F917F916F915F914F9166
:104A90003F912F910F900FBE0F901F9018951F926E
:104AA0000F920FB60F9211242F938F939F93EF9332
:104AB000FF93E091A004F091A1048081E091A6040D
:104AC000F091A70482FD1BC090818091A9048F5FA3
:104AD0008F732091AA04821741F0E091A904F0E0BD
:104AE000E057FB4F958F8093A904FF91EF919F9121
:104AF0008F912F910F900FBE0F901F90189580816E
:104B0000F4CF1F920F920FB60F9211242F933F9361
:104B10008F939F93AF93BF9380910404909105046A
:104B2000A0910604B09107043091030423E0230F01
:104B30002D3758F50196A11DB11D209303048093D4
:104B4000040490930504A0930604B0930704809195
:104B5000080490910904A0910A04B0910B040196F5
:104B6000A11DB11D8093080490930904A0930A0429
:104B7000B0930B04BF91AF919F918F913F912F9173
:104B80000F900FBE0F901F90189526E8230F0296E6
:104B9000A11DB11DD2CF1F920F920FB60F921124FB
:104BA0002F933F934F935F936F937F938F939F9335
:104BB000AF93BF93EF93FF938091B900887F8036C6
:104BC00009F44AC0F0F5883209F4A7C018F580311D
:104BD00009F49BC0B8F4882309F4F9C0883009F4BB
:104BE00094C0FF91EF91BF91AF919F918F917F9171
:104BF0006F915F914F913F912F910F900FBE0F904A
:104C00001F901895883109F488C0803251F780933D
:104C1000640414C0803409F49DC040F48033B9F3B7
:104C20008833F9F68093640485ECB0C0803509F4CC
:104C300085C0883509F496C0883499F60E947712A9
:104C4000D0CF883909F48CC038F5883729F050F472
:104C5000883611F0803729F683E08093660410923D
:104C6000020457C0883809F47BC0803919F08038B5
:104C700009F0B7CF80910204803208F071C0E09152
:104C8000020481E08E0F809302048091BB00F0E06B
:104C9000EE51FC4F80833DC0803B39F0E0F4803A18
:104CA00009F479C0883A09F09CCF84E080936604C7
:104CB0001092E1031092E003E0911C04F0911D04B6
:104CC00009958091E00381110FC081E08093E0039A
:104CD0001092C00309C0803C09F4A6CF883C09F4B7
:104CE000A3CF883B09F07DCFE091E10381E08E0FF7
:104CF0008093E103F0E0E054FC4F80818093BB009F
:104D00009091E1038091E00329C080914104809358
:104D1000BB0085EC8093BC0064CF909163048091CC
:104D20006204981758F5E091630481E08E0F809338
:104D30006304F0E0EE5BFB4F8081E9CFE091630418
:104D400081E08E0F809363048091BB00F0E0EE5B06
:104D5000FB4F808390916304809162049817C8F29E
:104D600085E8D8CFE091630481E08E0F80936304DF
:104D70008091BB00F0E0EE5BFB4F80838091650487
:104D800081115CCF81E08093400484EA8093BC0071
:104D90001092660426CF85EC8093BC0010926604C6
:104DA00080910204803230F4E0910204F0E0EE5190
:104DB000FC4F10826091020470E0E0911A04F091BF
:104DC0001B0482EE93E00995109202040ACF109220
:104DD000640434CFCF93DF93109293041092920423
:104DE00088EE93E0A0E0B0E0809394049093950463
:104DF000A0939604B093970426E331E03093910496
:104E00002093900425EC30E030939D0420939C0483
:104E100024EC30E030939F0420939E0420EC30E09B
:104E20003093A1042093A00421EC30E03093A3043C
:104E30002093A20422EC30E03093A5042093A40434
:104E400026EC30E03093A7042093A6041092A90426
:104E50001092AA041092AB041092AC041092300588
:104E600010922F058093310590933205A09333055E
:104E7000B093340588E491E090932E0580932D053E
:104E800010922306109222068AE591E09093210663
:104E90008093200610925B0610925C0610925D06CD
:104EA000109229061092280610922B0610922A06BC
:104EB00010922D0681E080932C0682E280932E06CC
:104EC0001092330610923206E7E4F6E085E596E0AC
:104ED000CFEFC1938E179F07E1F7D1E0D09344063F
:104EE00083E993E090933A0680933906D0933B068A
:104EF00010923C0610923D0680E480933E0610928C
:104F00003F0682E993E090935606809355068EE122
:104F100091E09093270680932606109252060E94F5
:104F2000F10A8AE591E09093210680932006109281
:104F30001F06C093ED05C093EE05C093EF05C09327
:104F4000F00564E671E08EED95E00E94661464E67B
:104F500071E088ED95E00E94661464E671E082EDF0
:104F600095E00E94661464E671E08CEC95E00E9486
:104F7000661464E671E086EC95E00E94661464E6CF
:104F800071E080EC95E00E94661464EC72E08AEBBC
:104F900095E00E9466146BEC72E084EB95E00E9451
:104FA000661410928D0585E080938E0510928F0512
:104FB000109291051092900510929305109292050F
:104FC000109294051092950565ED72E087E895E0E2
:104FD0000E94661486E190E090933A05809339052B
:104FE0008CE79CE8A1E0B0E08093450590934605EE
:104FF000A0934705B093480581EA97E6A3E3BDEB8C
:105000008093490590934A05A0934B05B0934C05B6
:1050100086E696E6A6EABFE380934D0590934E059B
:10502000A0934F05B0935005D093590589E190E0C6
:1050300090935B0580935A05D0935C0580E090E4E3
:10504000ACE1B5E480935D0590935E05A0935F05A8
:10505000B09360051092610510926205109263058D
:1050600010926405E5E6F5E080E1DF011D928A9586
:10507000E9F7109275051092760510927705109257
:1050800078051092790510927A0510927B0510929E
:105090007C0510927D0510927E0510927F0510927E
:1050A000800510928105109282051092830510925E
:1050B000840581E090E09093860580938505DF91DB
:1050C000CF910895CF93DF93CDB7DEB72C970FB66E
:1050D000F894DEBF0FBECDBF789484B5826084BDE6
:1050E00084B5816084BD85B5826085BD85B58160EC
:1050F00085BD80916E00816080936E00109281006A
:105100008091810082608093810080918100816024
:1051100080938100809180008160809380008091E5
:10512000B10084608093B1008091B0008160809371
:10513000B00080917A00846080937A0080917A0038
:10514000826080937A0080917A00816080937A00F7
:1051500080917A00806880937A001092C10061E0AB
:105160008EE00E947705E091A004F091A10482E016
:105170008083E0919C04F0919D041082E0919E0454
:10518000F0919F048FEC80831092A804E091A40416
:10519000F091A50486E08083E091A204F091A3043D
:1051A000808180618083E091A204F091A3048081DA
:1051B00088608083E091A204F091A30480818068DC
:1051C0008083E091A204F091A30480818F7D80838D
:1051D00060E08EE00E9449050E94480781E08093CC
:1051E0006C0483E280938E0410926D0410928F04FD
:1051F00060E18DE295E00E948D090E9480078FE3B7
:105200009CE90197F1F700C0000068EC70E080E0D5
:1052100090E00E94E80584E690E090931901809365
:1052200018010E94263280930C0485E690E00E94CB
:10523000263280930D0400910C0410910D04B801E6
:10524000012E000C880B990B0E9406319B01AC01CA
:105250000E949434811106C00B5011090C301105C5
:1052600008F436C184E690E00E94EF163DE8C32EB4
:1052700035E0D32E56010EE110E0C8010E9426321F
:10528000F50181935F010F5F1F4F07321105A9F7E9
:1052900010918E05612F012E000C770B880B990B56
:1052A0000E9406319B01AC010E949434811103C01D
:1052B000153009F438C18EE190E00E94181768ECAF
:1052C00070E080E090E00E94E80561EE72E08EED13
:1052D00095E00E9410140E94480764E670E080E0A8
:1052E00090E00E94E80565E671E0CE0101960E941B
:1052F0006614CE0101960E94D314CE0101960E943D
:1053000020138091260690912706F1E08F309F07A9
:1053100051F090931201809311018FE091E09093EE
:105320002706809326068FE29AE0909310018093DF
:105330000F0184E296E00E94CF0A6EED75E0CE0187
:1053400001960E945D146AEB75E0CE0107960E94FB
:105350005D1448EE53E0BE016F5F7F4FCE010796AC
:105360000E94A015CE0107960E942013CE0101963F
:105370000E9420136AEB75E0CE0101960E945D1435
:10538000CE0101960E947C13BC018EED95E00E9437
:10539000C313CE0101960E9420136EED75E0CE017D
:1053A00001960E945D14CE0101960E94D314CE0195
:1053B00001960E94201386E78093E4058091ED0515
:1053C0008F3F11F40E9448078091ED058F3F01F552
:1053D0008091E40591E090936C0480938E04109288
:1053E0006D0410928F0460ED8DE295E00E948D09AE
:1053F0000E94800761E08091E4050E946708109296
:105400001F0480931E048DE295E00E944609F82E49
:1054100028E5F21609F495C06AEE72E08EED95E08B
:105420000E941014109215016EED75E0CE010196E8
:105430000E945D14CE0101960E94D314CE01019604
:105440000E9420138AE2C82ED12C98EE892E93E078
:10545000992EA12CB12C20E0E22E20E0F22E01E0CA
:1054600064E671E0CE0107960E94661410E080E9C0
:1054700094E00E944D04181619060CF0D3C01111C7
:10548000D1C080E994E00E942B048A3009F07AC1EF
:1054900010910E04112309F48AC18091D0059091D6
:1054A000D105892B09F47CC166EF72E0CE0101962B
:1054B0000E946614BE01695F7F4FCE0101960E9473
:1054C000B0130E940304CE0101960E94201368C10C
:1054D00049E3C42E45E0D42E04E610E0C8010E9442
:1054E0002632F60181936F010F5F1F4F023B1105BA
:1054F000A9F78091390590913A059093170180930F
:1055000016016BE375E0CE0101960E946614BE01A0
:105510006F5F7F4F8AEB95E00E94D512CE01019616
:105520000E942013A3CE0EE110E0C8010E94263293
:10553000F60181936F010F5F1F4F05341105A9F725
:10554000BECE88E80E940C129093F2058093F1057C
:105550008AE80E940C129093F4058093F3058CE87E
:105560000E940C129093F6058093F5058EE80E9438
:105570000C129093F8058093F70580E90E940C12B5
:105580009093FA058093F90582E90E940C1290939A
:10559000FC058093FB0584E90E940C129093FE05A4
:1055A0008093FD0586E90E940C129093000680937B
:1055B000FF0588E90E940C12909302068093010671
:1055C0008AE90E940C1290930406809303068CE9EA
:1055D0000E940C1290930606809305068EE90E94A5
:1055E0000C1290930806809307068091ED058F3F7B
:1055F00009F028CF8091E40591E090936C048093AA
:105600008E0410926D0410928F0464EF8DE295E089
:105610000E948D096FE38DE295E00E948D090E9442
:10562000800710CF8B859C85892B51F080E994E011
:105630000E94DC0464E170E080E090E00E94E805F4
:10564000BE01695F7F4F8CEC95E00E94D512CE01C0
:1056500007960E94201364E671E08EED95E00E94AB
:1056600010148091D0059091D1058130910509F0F9
:10567000C6C06CEC75E088ED95E00E9446140E946F
:10568000601268ED75E0CE0101960E945D148D8177
:105690009E81892B09F4A5C0E981FA81309709F42C
:1056A000A0C08081823409F484C0833409F48EC0A0
:1056B000813409F096C06FEF72E08CEC95E00E94A7
:1056C0001014CE0101960E9420138CEC95E00E94EC
:1056D000AF12CB010E94ED1D80911704882309F4BD
:1056E0003FC00E94F706A50194010E94A532CA019D
:1056F000B9010E94043120911304309114044091A7
:105700001504509116040E94D63220911A0130914E
:105710001B0140911C0150911D010E943F3418163D
:10572000FCF480911104909112044A9609F4BFC0D0
:1057300080910F04909110040E94ED1D0E94F706C5
:10574000A50194010E94A532CA01B9010E94043149
:1057500060931304709314048093150490931604BB
:105760006AE070E080E090E00E94E805E114F10456
:1057700009F476CE0E945904882309F471CE0E9460
:1057800000006ECE8D3009F483CE89831A8241E009
:1057900050E0BE016F5F7F4FCE0107960E9450130D
:1057A0006AE070E080E090E00E94E80560CE11E0E1
:1057B000F7CF62E073E08CEC95E00E941014109239
:1057C00017048CEF9FEF0E94ED1D7BCF65E073E027
:1057D0008CEC95E00E941014009317048DEF9FEF5E
:1057E000F2CFBE016F5F7F4F8CEC95E00E944614B4
:1057F0006AE070E080E090E00E94E80562CF0497E4
:1058000068F568EE71E0CE0101960E946614BE0153
:105810006F5F7F4F8CEC95E00E94BA12182FCE017B
:1058200001960E9420131123C9F08091D005909118
:10583000D105029788F0E091CC05F091CD05309725
:1058400059F0818180330CF4845EF601E81BF10984
:1058500087FDF395CF013ECF80E0F6CF6CEC75E08D
:1058600088ED95E00E9446140E9460121A82198207
:105870001C821B821E821D8261E876E0CE010196A9
:105880000E94CA13BE016F5F7F4F88ED95E00E94B2
:10589000BA12182FCE0101960E942013112321F075
:1058A000F0E0E0E0099518CF0E94411715CF8091F4
:1058B0008D05882309F442CF0E9405253FCF87E854
:1058C00095E00E94201384EB95E00E9420138AEB60
:1058D00095E00E94201380EC95E00E94201386EC56
:1058E00095E00E9420138CEC95E00E94201382ED3D
:1058F00095E00E94201388ED95E00E9420138EED24
:1059000095E00C942013EF920F931F93CF93DF93A6
:10591000E80134E047FD34E1042E000C550B57FF3D
:1059200003C0519541955109E32E022F242FAE015A
:105930000E94472DCE01DF91CF911F910F91EF90E3
:105940000895662777270C94A62E1F93FC019927AC
:105950008827BC01E89411911032E9F3193010F056
:105960001E30C8F31B3251F01D3249F4689406C052
:105970000E94F62C610F711D811D911D1191105314
:105980001A30B0F33EF490958095709561957F4FF5
:105990008F4F9F4F1F910895FB01DC0105900D92E1
:1059A0000020E1F70895FC0105900020E9F78095BB
:1059B00090958E0F9F1F0895BB274A3031F499238D
:1059C00022F4BDE2909581959F4F0C942E2DBB271C
:1059D0002A3051F4992342F4BDE290958095709558
:1059E00061957F4F8F4F9F4F0C940C2D592F482F4F
:1059F000372F262F660F771F881F991F660F771F77
:105A0000881F991F620F731F841F951F660F771FD2
:105A1000881F991F0895BB27FA01A62F62177105E9
:105A200081059105330B30FB66F0AA27660F771FBF
:105A3000881F991FAA1FA21710F0A21B6395385048
:105A4000A9F7A05DAA3308F0A95DA19336F7B111BB
:105A5000B1931082CA010C94EF30BB27FB0155278C
:105A6000AA27880F991FAA1FA41710F0A41B8395BB
:105A70005051B9F7A05DAA3308F0A95DA193009732
:105A800079F7B111B1931192CB010C94EF30A9E0E9
:105A9000B0E0EDE4FDE20C9474326A01F22EB02E17
:105AA000102FFBE3AF2EA01608F41BE31F5F012F9E
:105AB00027E0AE014F5F5F4F0E94F62FBC01898146
:105AC000982F9970913009F43FC09BE2E1FC04C02B
:105AD0009E2D9170E0FC3AC05E2D5071E82FE87069
:105AE00083FF46C084E0911101C083E0EF2DE81BE5
:105AF0008F1508F0E0E0D6018E2F20E2552351F1FA
:105B0000992329F0D6019C93C60101966C01960158
:105B10002D5F3F4FE2FE24C08EE4D6018C9391E4CA
:105B200011969C93119712968C93D9018E2F90E227
:105B300081111BC0E20FF32FF11D10828EEF9FEF3A
:105B40002996ECE00C9490329DE2C6CF90E2C4CF4F
:105B50002D9381508111FCCFCE0ED11CE0E0D0CF2F
:105B60008EE6D6018C9391E6DBCF9D938150E0CFFA
:105B7000482F447082FF3DC084E0911101C083E052
:105B80008F1510F4EF2DE81BD6018E2F20E2552340
:105B900009F1992329F0D6019C93C60101966C0165
:105BA00096012D5F3F4FE2FE1BC089E4D6018C9326
:105BB0008EE411968C93119786E412968C93D901FA
:105BC0008E2F90E2882309F4B5CF9D938150FACFB0
:105BD0002D9381508111FCCFCE0ED11CE0E0D9CFA6
:105BE00089E6D6018C938EE611968C93119786E602
:105BF000E4CF9B0177FF02C030E020E0A1E0B0E0FD
:105C0000911102C0B0E0A0E0F9013196AE0FBF1FC4
:105C10008B2C912CBB2009F461C05401EFEFAE1A1C
:105C2000BE0AAA0DBB1DFA161B0619F014F04F2D63
:105C30004A1B511188C0E3FC59C07601A42FB0E281
:105C4000A1114FC0C40ED11C992309F45BC040E0E0
:105C5000D6011196F60190836D01552309F448C0D1
:105C6000012F060F9A81582F507184FF03C0913382
:105C700009F4015010160CF047C0093008F008E094
:105C8000EEE2FE2E5B01A01AB10885019194819489
:105C900091082F3F320729F4D601FC92F601319684
:105CA0006F016217730794F1021713077CF5DB018C
:105CB000A21BB30BAA24A394B12CAC0EBD1EAA0D3B
:105CC000BB1D11968C9121503109D60111962815D2
:105CD0003905F4F0F60180836D01DBCFB12CA12CE6
:105CE000A0CFF701B1937F01A150AACF9111B0CFFE
:105CF000D601942F50E302C05D9391509111FCCFD7
:105D0000C40ED11C40E0ACCF01E0BACF80E3DBCFC2
:105D10006217730731F4963388F4953311F45523E1
:105D200069F0F6018083FD01842F90E2811108C0A3
:105D3000A40FB11D1C9290E080E002CF81E3F1CF6F
:105D400091938150F3CF911183CF8ACFB0E0A0E03F
:105D5000ECEAFEE20C9474325C017B016115710582
:105D600019F0DB018D939C9385010F5F1F4FF501A7
:105D7000D0818D2F90E00E94CE306C01892BB9F537
:105D8000DD32B9F50F5F1F4FD5011196DC91C1E0EF
:105D90005801F1E0AF1AB10843E050E062EF70E063
:105DA000C5010E94D730892B69F5680182E0C80ED1
:105DB000D11C45E050E06DEE70E0C6010E94D73086
:105DC000892B21F4680197E0C90ED11CE114F1047C
:105DD00019F0D701CD92DC9260E070E080E89FEF8F
:105DE000C111FFC060E070E080E89FE7FAC0580191
:105DF000BBCFDB3229F485010E5F1F4FF501D18146
:105E0000C0E0C6CF43E050E06AEE70E0C5010E94FA
:105E1000D730892BE9F0F80110E000E020E030E015
:105E2000A9015F01B0ED8B2E8D0E89E08815C8F1B8
:105E30009C2E689491F88C2F8870C2FF16C0811137
:105E400002C00F5F1F4F3196D501DC91C92DE9CFFC
:105E5000E114F10429F00E5F1F4FF7011183008355
:105E600060E070E080EC9FE7BCC0882311F0015037
:105E70001109A5E0B0E00E945B329B01AC01220F4A
:105E8000331F441F551F280D311D411D511D283939
:105E900099E93907490799E15907A8F2C6609C2E8C
:105EA000D2CFAEEF8A1206C0C3FD3CC09C2E6894D0
:105EB00093F8C9CFDF7DD534A9F580818D3239F4CF
:105EC000C061DF011296818162E070E006C0DF01EF
:105ED0008B32C1F3119661E070E080535D01A61A28
:105EE000B70A8A30F8F4E0E8CE16ECE0DE065CF49F
:105EF000B601660F771F660F771FC60ED71ECC0C34
:105F0000DD1CC80ED11C5D01FFEFAF1ABF0A8C91DA
:105F100080538A30A8F1C4FF03C0D194C194D10842
:105F20000C0D1D1DC1FF09C0E114F10431F081E029
:105F3000A81AB108D701AD92BC92CA01B9010E945A
:105F40000431C370C33009F490584B015C0120E068
:105F500030E0A9010E94FF30882309F440C0C1E26B
:105F6000D1E017FF05C0119501951109C9E0D1E0F5
:105F70006E01B8E1CB1AD10880E2E82EF12C0FC0F7
:105F8000D501B1CFFE0125913591459154910E195E
:105F90001F09C501B4010E9465314B015C01D501A7
:105FA000C4010E151F0574F72497F594E794CC16D9
:105FB000DD06A9F78A2F880F8B2F881F8F3F49F0A6
:105FC00020E030E0A901C501B4010E94FF30811139
:105FD00006C082E290E090935F0680935E06C50162
:105FE000B401CDB7DEB7ECE00C949032283008F065
:105FF00027E03327DA01990F311D87FD9160009664
:106000006105710539F432602E5F3D9330E32A95C6
:10601000E1F708959F3F30F080387105610509F080
:106020003C5F3C5F3D93913008F08068911DDF93A9
:10603000CF931F930F93FF92EF92192F987F96950E
:10604000E92F96959695E90FFF27E158FE4F99277E
:106050003327EE24FF24A701E70105900894079455
:1060600028F4360FE71EF81E491F511D660F771FD3
:10607000881F991F0694A1F70590079428F4E70E4E
:10608000F81E491F561FC11D770F881F991F661FD5
:106090000694A1F70590079428F4F80E491F561F9F
:1060A000C71FD11D880F991F661F771F0694A1F780
:1060B0000590079420F4490F561FC71FD81F990F4A
:1060C000661F771F881F0694A9F784911095177093
:1060D00041F0D695C79557954795F794E7941A954B
:1060E000C1F7E5E2F1E0689415901591359165915D
:1060F000959105907FE27395E118F10A430B560BD9
:10610000C90BD009C0F7E10CF11E431F561FC91F70
:10611000D01D7EF4703311F48A95E6CFE8940150D7
:1061200030F0080F0AF40027021708F4202F2395F7
:10613000022F7A3328F079E37D932A95E9F710C08E
:106140007D932A9589F606949795679537951795C7
:106150001794E118F10A430B560BC90BD00998F0BC
:1061600023957E9173957A3308F070E37C93201326
:10617000B8F77E9170617D9330F0839571E37D93E4
:1061800070E32A95E1F71124EF90FF900F911F9192
:10619000CF91DF91992787FD9095089591110C94E7
:1061A000D231803219F089508550C8F70895FB012B
:1061B000DC014150504088F08D9181341CF08B35CA
:1061C0000CF4805E659161341CF06B350CF4605EFC
:1061D000861B611171F3990B0895881BFCCFDC01BC
:1061E000FC01672F71917723E1F7329704C07C910E
:1061F0006D9370836291AE17BF07C8F308950E9434
:10620000413108F481E00895E89409C097FB3EF419
:1062100090958095709561957F4F8F4F9F4F9923F3
:10622000A9F0F92F96E9BB279395F6958795779571
:106230006795B795F111F8CFFAF4BB0F11F460FF31
:106240001BC06F5F7F4F8F4F9F4F16C0882311F089
:1062500096E911C0772321F09EE8872F762F05C09D
:10626000662371F096E8862F70E060E02AF09A9538
:10627000660F771F881FDAF7880F9695879597F92D
:106280000895990F0008550FAA0BE0E8FEEF1616C7
:106290001706E807F907C0F012161306E407F5071A
:1062A00098F0621B730B840B950B39F40A2661F08E
:1062B000232B242B252B21F408950A2609F4A14031
:1062C000A6958FEF811D811D08950E9478310C9451
:1062D000EC310E94DE3138F00E94E53120F0952348
:1062E00011F00C94D5310C94DB3111240C94203234
:1062F0000E94FD3170F3959FC1F3950F50E0551F3B
:10630000629FF001729FBB27F00DB11D639FAA270A
:10631000F00DB11DAA1F649F6627B00DA11D661F59
:10632000829F2227B00DA11D621F739FB00DA11D7A
:10633000621F839FA00D611D221F749F3327A00D34
:10634000611D231F849F600D211D822F762F6A2FD0
:1063500011249F5750409AF0F1F088234AF0EE0F35
:10636000FF1FBB1F661F771F881F91505040A9F762
:106370009E3F510580F00C94D5310C9420325F3F44
:10638000E4F3983ED4F3869577956795B795F7959E
:10639000E7959F5FC1F7FE2B880F911D9695879516
:1063A00097F9089599278827089597F99F6780E8B6
:1063B00070E060E008959FEF80EC089500240A9457
:1063C0001616170618060906089500240A941216D0
:1063D0001306140605060895092E0394000C11F403
:1063E000882352F0BB0F40F4BF2B11F460FF04C0B0
:1063F0006F5F7F4F8F4F9F4F089557FD9058440F09
:10640000551F59F05F3F71F04795880F97FB991F13
:1064100061F09F3F79F087950895121613061406D0
:10642000551FF2CF4695F1DF08C01616170618065D
:10643000991FF1CF86957105610508940895E89438
:10644000BB2766277727CB0197F90895F999FECFE7
:1064500092BD81BDF89A992780B50895262FF999A4
:10646000FECF1FBA92BD81BD20BD0FB6F894FA9A37
:10647000F99A0FBE01960895052E97FB1EF400941D
:106480000E94533257FD07D00E94A53207FC03D06B
:106490004EF40C94533250954095309521953F4FD2
:1064A0004F4F5F4F089590958095709561957F4F00
:1064B0008F4F9F4F08950E94C732A59F900DB49FA4
:1064C000900DA49F800D911D11240895B7FF0C9489
:1064D0005B320E945B32821B930B08952F923F9296
:1064E0004F925F926F927F928F929F92AF92BF92E4
:1064F000CF92DF92EF92FF920F931F93CF93DF9390
:10650000CDB7DEB7CA1BDB0B0FB6F894DEBF0FBEEC
:10651000CDBF09942A88398848885F846E847D8439
:106520008C849B84AA84B984C884DF80EE80FD803B
:106530000C811B81AA81B981CE0FD11D0FB6F894B1
:10654000DEBF0FBECDBFED010895A1E21A2EAA1B3A
:10655000BB1BFD010DC0AA1FBB1FEE1FFF1FA21713
:10656000B307E407F50720F0A21BB30BE40BF50B10
:10657000661F771F881F991F1A9469F76095709599
:10658000809590959B01AC01BD01CF010895A29F1C
:10659000B001B39FC001A39F700D811D1124911DF7
:1065A000B29F700D811D1124911D08955058BB2775
:1065B000AA270E94EE320C94EC310E94DE3138F0B2
:1065C0000E94E53120F039F49F3F19F426F40C9431
:1065D000DB310EF4E095E7FB0C94D531E92F0E94F6
:1065E000FD3158F3BA17620773078407950720F047
:1065F00079F4A6F50C941F320EF4E0950B2EBA2F09
:10660000A02D0B01B90190010C01CA01A0011124B8
:10661000FF27591B99F0593F50F4503E68F11A1664
:10662000F040A22F232F342F4427585FF3CF4695F5
:1066300037952795A795F0405395C9F77EF41F1617
:10664000BA0B620B730B840BBAF09150A1F0FF0FE1
:10665000BB1F661F771F881FC2F70EC0BA0F621FCD
:10666000731F841F48F4879577956795B795F795BD
:106670009E3F08F0B0CF9395880F08F09927EE0F52
:106680009795879508950E9457330C94EC310E949A
:10669000E53158F00E94DE3140F029F45F3F29F0E7
:1066A0000C94D53151110C9420320C94DB310E94A2
:1066B000FD3168F39923B1F3552391F3951B550BE5
:1066C000BB27AA2762177307840738F09F5F5F4FC5
:1066D000220F331F441FAA1FA9F335D00E2E3AF004
:1066E000E0E832D091505040E695001CCAF72BD01C
:1066F000FE2F29D0660F771F881FBB1F261737076D
:106700004807AB07B0E809F0BB0B802DBF01FF279E
:1067100093585F4F3AF09E3F510578F00C94D53175
:106720000C9420325F3FE4F3983ED4F3869577953E
:106730006795B795F7959F5FC9F7880F911D969557
:10674000879597F90895E1E0660F771F881FBB1FB3
:10675000621773078407BA0720F0621B730B840B60
:10676000BA0BEE1F88F7E09508950E94BC33689439
:10677000B1110C94203208950E94053288F09F5781
:1067800098F0B92F9927B751B0F0E1F0660F771F55
:10679000881F991F1AF0BA95C9F714C0B13091F04B
:1067A0000E941F32B1E008950C941F32672F782F9A
:1067B0008827B85F39F0B93FCCF386957795679510
:1067C000B395D9F73EF490958095709561957F4F7C
:1067D0008F4F9F4F089597FB16F40E942F340C940F
:1067E000F233E894F92F96EBFF2381F0121613068B
:1067F0001406440B9395F69587957795679557956D
:106800004040FF23B9F71BC099270895882351F40E
:106810009850D2F7872B762F652F542F432F322F86
:1068200020E0B1F3121613061406440B88233AF045
:106830009A95440F551F661F771F881FCAF7552367
:106840004AF4440F551F11F460FF04C06F5F7F4F7F
:106850008F4F9F4F880F9695879597F9089590953C
:1068600080957095609550954095309521953F4F56
:106870004F4F5F4F6F4F7F4F8F4F9F4F08950E9435
:10688000413108F48FEF0895FA01EE0FFF1F3096A3
:1068900021053105A1F16115710561F48038BFE36F
:1068A0009B0749F168949038810561F08038BFEF0B
:1068B0009B0741F099234AF5FF3FE105310521058A
:1068C00019F1E8940894E795D901AA2329F4AB2F8C
:1068D000BE2FF85FD0F310C0FF5F70F4A695E0F70D
:1068E000F73950F019F0FF3A38F49F779F930DD0A5
:1068F0000F9007FC9058089546F00C94DB3160E04F
:1069000070E080E89FE308954FE79F775F934F9390
:106910003F932F930E9444352F913F914F915F9168
:106920000E9465310C94A1340E944131880B990B6F
:10693000089529F416F00C94D5310C941F320C9460
:10694000DB310E940532A8F39638A0F707F80F92C2
:10695000E8942BE33AEA48EB5FE70E947B310F9221
:106960000F920F924DB75EB70F920E948C35E8E6FA
:10697000F0E00E94D3344F915F91EF91FF91E59544
:10698000EE1FFF1F49F0FE57E0684427EE0F441F3B
:10699000FA95E1F74195550B0E9406350F9007FED9
:1069A0000C94FA340895DF93CF931F930F93FF92C3
:1069B000EF92DF927B018C01689406C0DA2EEF0122
:1069C0000E947831FE01E894A59125913591459179
:1069D0005591A6F3EF010E94EE32FE019701A80146
:1069E000DA9469F7DF90EF90FF900F911F91CF91AC
:1069F000DF9108959B01AC0160E070E080E89FE3C7
:106A00000C9443330C94D5310C94C0350E9405325C
:106A1000D8F39923C9F3940F511DA3F3915050401B
:106A200094F059F0882332F0660F771F881F915039
:106A30005040C1F79E3F51052CF7880F911D969548
:106A4000879597F908955F3FACF0983E9CF0BB277F
:106A5000869577956795B79508F4B1609395C1F7DA
:106A6000BB0F58F711F460FFE8CF6F5F7F4F8F4F78
:106A70009F4FE3CF0C94203216F00C94C0350C9449
:106A8000DB3168940C94D5310E940532A8F3992328
:106A9000C1F3AEF3DF93CF931F930F93FF92C92FF0
:106AA000DD2788232AF02197660F771F881FDAF7E2
:106AB00020E030E040E85FEB9FE3883920F0803E43
:106AC00038F021968F770E94D732E0E9F0E004C0D9
:106AD0000E94D732EDEBF0E00E94D3348B01BE016F
:106AE000EC01FB2E6F5771097595771F880B990B79
:106AF0000E94063128E132E741E35FE30E947831EA
:106B0000AF2D9801AE01FF900F911F91CF91DF91B2
:106B10000E94EE320C94EC31FA01DC01AA0FBB1F8B
:106B20009B01AC01BF5728F4222733274427507814
:106B300020C0B75190F4AB2F002446953795279588
:106B4000011CA395D2F3002071F0220F331F441FC4
:106B5000B395DAF30ED00C94D63261307105A0E80B
:106B60008A07B94630F49B01AC016627772788274E
:106B70009078309621F020833183428353830895A7
:106B80009F3F31F0915020F4879577956795B795A1
:106B9000880F911D9695879597F90895DB018F933E
:106BA0009F930E945B32BF91AF91A29F800D911D78
:106BB000A39F900DB29F900D11240895AA1BBB1B9B
:106BC00051E107C0AA1FBB1FA617B70710F0A61BED
:106BD000B70B881F991F5A95A9F780959095BC010E
:106BE000CD010895EE0FFF1F0590F491E02D09945B
:106BF000DF93CF931F930F939A9DF02D219FF00D5C
:106C00008B9DF00D8A9DE02DF10D039FF00D029FED
:106C1000E00DF11D4E9DE00DF11D5E9DF00D4F9DAF
:106C2000F00D7F936F93BF92AF925F934F93D50117
:106C30000E94C7328B01AC01D7010E94C732EB0121
:106C4000E80FF91FD6010E9447362F913F91D601D8
:106C50000E94C732C60FD71FE81FF91FAF91BF911F
:106C60000E9447362F913F910E94C732C60FD71F0F
:106C7000E81FF91FD6010E94C732E60FF71F9801DF
:106C8000BE01CF010F911F91CF91DF9108950E9416
:106C9000C732460F571FC81FD91F08F431960895F1
:106CA000689401C0E894F92FF12B12F00C9484360B
:106CB000A0E0B0E0EEE5F6E30C947432092E059402
:106CC00022F40E94E036112392F4F0E80F26FFEF41
:106CD000E094F09400951095B094C094D094A19451
:106CE000BF0ACF0ADF0AEF0AFF0A0F0B1F0B0E9431
:106CF0008F3607FC0E94E036CDB7DEB7ECE00C948F
:106D00009032689401C0E8948F929F92CF93DF9362
:106D10000E948F36DF91CF919F908F9008958824A5
:106D20009924F401E401B0E49F93AA279A158B04F7
:106D30009C04ED05FE05CF05D007A10798F4AD2F03
:106D4000DC2FCF2FFE2FE92D982C892E982F872FFF
:106D5000762F652F542F432F322F2227B85031F72B
:106D6000BF9127C01B2EBF91BB27220F331F441F8B
:106D7000551F661F771F881F991F881C991CEE1FBF
:106D8000FF1FCC1FDD1FAA1FBB1F8A149B04EC052D
:106D9000FD05CE05DF05A007B10748F08A189B085E
:106DA000EC09FD09CE09DF09A00BB10B21601A9493
:106DB000E1F62EF49401AF01BE01CD01000C08955F
:106DC000609570958095909530954095509521955A
:106DD0003F4F4F4F5F4F6F4F7F4F8F4F9F4F0895E4
:106DE000002E083090F0982F872F762F652F542F84
:106DF000432F322F22270850F4CF220F331F441F76
:106E0000551F661F771F881F991F0A95B2F7002D1F
:106E1000089597FD1094002E083098F00850232F05
:106E2000342F452F562F672F782F892F912DF4CF90
:106E300015949795879577956795579547953795C5
:106E400027950A95AAF71124002D08952A0D3B1DB8
:106E50004C1D5D1D6E1D7F1D801F911F08952A19F9
:106E60003B094C095D096E097F09800B910B089560
:106E70000024A7FD00942A17300540055005600541
:106E800070058005900508950F931F93CF93DF93AE
:106E90008230910510F482E090E0E0916206F0917A
:106EA000630630E020E0B0E0A0E0309799F42115CF
:106EB000310509F44AC0281B390B24303105D8F5B7
:106EC0008A819B816115710589F1FB01938382831E
:106ED000FE0111C040815181028113814817590779
:106EE000E0F04817590799F4109761F012960C9347
:106EF000129713961C933296CF01DF91CF911F9179
:106F00000F9108950093620610936306F4CF211544
:106F1000310551F04217530738F0A901DB019A01FE
:106F2000BD01DF01F801C1CFEF01F9CF90936306F6
:106F300080936206CDCFFE01E20FF31F8193919300
:106F40002250310939832883D7CF209160063091B0
:106F50006106232B41F420912601309127013093C3
:106F600061062093600620912401309125012115AE
:106F7000310541F42DB73EB74091280150912901C8
:106F8000241B350BE0916006F0916106E217F307D0
:106F9000A0F42E1B3F0B2817390778F0AC014E5F89
:106FA0005F4F2417350748F04E0F5F1F509361065F
:106FB00040936006819391939FCFF0E0E0E09CCFF7
:106FC000CF93DF930097E9F0FC013297138212828E
:106FD000A0916206B0916306ED0130E020E01097C9
:106FE000A1F420813181820F931F2091600630919E
:106FF00061062817390709F061C0F0936106E09334
:107000006006DF91CF910895EA01CE17DF07E8F51A
:107010004A815B819E0141155105B1F7E901FB836E
:10702000EA8349915991C40FD51FEC17FD0761F40C
:10703000808191810296840F951FE901998388834D
:10704000828193819B838A83F0E0E0E012968D91A8
:107050009C9113970097B9F52D913C911197CD0113
:107060000296820F931F20916006309161062817C7
:10707000390739F6309751F510926306109262067F
:10708000B0936106A0936006BCCFD383C2834081D6
:107090005181840F951FC817D90761F44E5F5F4F68
:1070A00088819981480F591F518340838A819B8130
:1070B000938382832115310509F0B0CFF0936306E5
:1070C000E09362069ECFFD01DC01C0CF13821282E5
:1070D000D7CFB0E0A0E0EFE6F8E30C9470328C017B
:1070E000009751F4CB010E9444378C01C801CDB701
:1070F000DEB7E0E10C948C32FC01E60FF71F9C0137
:1071000022503109E217F30708F49DC0D901CD914F
:10711000DC911197C617D70798F0C530D10530F329
:10712000CE0104978617970708F3C61BD70B229743
:10713000C193D1936D937C93CF010E94E037D6CF5A
:107140005B01AC1ABD0A4C018C0E9D1EA09162061B
:10715000B0916306512C412CF12CE12C109731F5A4
:1071600080916006909161068815990509F05CC0D0
:107170004616570608F058C08091240190912501C9
:10718000009741F48DB79EB7409128015091290195
:10719000841B950BE817F90708F055C0F0936106BA
:1071A000E0936006F90171836083A0CF8D919C917B
:1071B000119712966C90129713967C901397A815BE
:1071C000B90559F56C0142E0C40ED11CCA14DB04A8
:1071D00020F1AC014A195B09DA011296159780F08B
:1071E0006282738251834083D9016D937C93E11451
:1071F000F10471F0D7011396FC93EE93129776CFBA
:1072000022968C0F9D1FF90191838083F301EFCFAC
:10721000F0936306E093620669CF4816590608F4B6
:107220002C017D01D3019ACFCB010E9444377C0110
:10723000009749F0AE01B8010E942E39C8010E94A2
:10724000E037870153CF10E000E050CF911108954F
:1072500081568A5108F4805285580895FB01DC015B
:1072600002C001900D9241505040D8F70895FB01A3
:10727000DC0101900D920020E1F70895FB01DC0193
:107280004150504030F08D910190801919F4002048
:10729000B9F7881B990B0895FB01DC014150504060
:1072A00048F001900D920020C9F701C01D92415095
:1072B0005040E0F70895FB0151915523A9F0BF011B
:1072C000DC014D9145174111E1F759F4CD010190D1
:1072D000002049F04D9140154111C9F3FB014111C6
:1072E000EFCF81E090E00197089513E0C7E6D3E087
:1072F00004C0FE010E94F2352196C836D107C9F7B5
:10730000F894FFCF08200000008008030000A04090
:10731000C80001BC09000000000116006400000064
:10732000F041E50D00010E0D000064068000000133
:1073300000FF0100FF00000000008F04D6031C04C2
:10734000DC044D042B043F04000000008D0960099B
:10735000230F360959094609370900000000FC0EC1
:10736000D603230FD5030D0A002020202020202043
:1073700020202020202020002356657273696F6E24
:107380003A00234C6F67676572204E616D653A0065
:1073900053484F57533D0047455400732000534115
:1073A00056453D0054494D45493D0023496E74659D
:1073B0007276616C3D0054494D45443D002344754F
:1073C000726174696F6E3D004448543D0042543D03
:1073D00000534C20503D00506120756E6C696B6508
:1073E0006C792100685061004950414444002349B0
:1073F000503A004E45543D0055565A0023555620EC
:1074000056303D005620004D533D002C0023496E60
:10741000636F727265637421204D533D3132334482
:107420003344350020572F6D5E3200555620496E8B
:1074300074656E7369747900572F6D5E3220005544
:10744000563D006F432000250054656D702048753F
:107450006D696469747900483D0068506120006F6F
:1074600043006D0020413D004C6967687420496EFF
:1074700074656E7369747900206C7820004C3D004F
:10748000495220466C616D65204C6576656C3D0007
:10749000476173206C6576656C3D00204D756C749A
:1074A0006973656E736F72730023456E61626C65FC
:1074B000002344697361626C650023496E76616CD8
:1074C0006964206B65792100424E4D4C3033004E8B
:1074D000616E6F423268365000234E6F2053656EE6
:1074E000736F72210057656C636F6D653A0023629C
:1074F0006D70206661696C65640073657269616CAA
:0C7500003A20002D35002D34002D330002
:107E0000112484B714BE81FFF0D085E080938100F7
:107E100082E08093C00088E18093C10086E0809377
:107E2000C20080E18093C4008EE0C9D0259A86E02C
:107E300020E33CEF91E0309385002093840096BBD3
:107E4000B09BFECF1D9AA8958150A9F7CC24DD24C4
:107E500088248394B5E0AB2EA1E19A2EF3E0BF2EE7
:107E6000A2D0813461F49FD0082FAFD0023811F036
:107E7000013811F484E001C083E08DD089C08234E0
:107E800011F484E103C0853419F485E0A6D080C0E4
:107E9000853579F488D0E82EFF2485D0082F10E0AE
:107EA000102F00270E291F29000F111F8ED06801E7
:107EB0006FC0863521F484E090D080E0DECF843638
:107EC00009F040C070D06FD0082F6DD080E0C81688
:107ED00080E7D80618F4F601B7BEE895C0E0D1E017
:107EE00062D089930C17E1F7F0E0CF16F0E7DF06D8
:107EF00018F0F601B7BEE89568D007B600FCFDCFD4
:107F0000A601A0E0B1E02C9130E011968C91119780
:107F100090E0982F8827822B932B1296FA010C0160
:107F200087BEE89511244E5F5F4FF1E0A038BF0790
:107F300051F7F601A7BEE89507B600FCFDCF97BE46
:107F4000E89526C08437B1F42ED02DD0F82E2BD052
:107F50003CD0F601EF2C8F010F5F1F4F84911BD097
:107F6000EA94F801C1F70894C11CD11CFA94CF0C13
:107F7000D11C0EC0853739F428D08EE10CD085E9AC
:107F80000AD08FE07ACF813511F488E018D01DD067
:107F900080E101D065CF982F8091C00085FFFCCF94
:107FA0009093C60008958091C00087FFFCCF809118
:107FB000C00084FD01C0A8958091C6000895E0E648
:107FC000F0E098E1908380830895EDDF803219F02E
:107FD00088E0F5DFFFCF84E1DECF1F93182FE3DFCA
:107FE0001150E9F7F2DF1F91089580E0E8DFEE27F6
:047FF000FF270994CA
:027FFE00040479
:00000001FF
